:020000040000FA
:0608000002EF4BF01200B4
:0608080096EF3DF0120026
:06082A000B00E096000047
:10083000B90300000A000000DE960000E10300009A
:1008400002000000DA960000D70300000400000058
:10085000B496000026030000260000006396000006
:1008600000010000510000003D9600000003000060
:10087000260000003B960000DF030000020000009D
:10088000389600005D0F0000030000002B7B000085
:10089000FF02000001000000289600008503000010
:1008A0001000000026960000DD030000020000009A
:1008B0000B01006B0A0E005D2BE20051240DF3CFFB
:1008C00001FBF4CF02FB000E01270C0E022385EC86
:1008D0000EF00A0EEF6EECEC0FF0EF90ECEC0FF078
:1008E000EF82ECEC0FF0EF84ECEC0FF0EF98ECEC17
:1008F0000FF0EF9685EC0EF09CEC0FF085EC0EF00F
:10090000C0EC0FF085EC0EF0D0EC0FF0002BD2D73E
:1009100012000B01006B0A0E005D3FE20051240D36
:10092000F3CF01FBF4CF02FB000E01270C0E0223D4
:1009300071EC0EF0EF500A082EE171EC0EF0EF6A48
:1009400071EC0EF00B0E53C1EBFF0C0E54C1EBFF1C
:1009500071EC0EF00D0EEB6A0E0EEB6A71EC0EF000
:10096000CBEC0FF00CEC10F0EF800CEC10F0EF96ED
:1009700071EC0EF0AEEC0EF008E071EC0EF07FECD6
:100980000EF071EC0EF09CEC0FF00CEC10F0EF821E
:100990000B0100511200002BBED7FE0C0B016F6B38
:1009A0006C6B0A0E6C5D14E26C51240DF3CF6DFB81
:1009B000F4CF6EFB000E6D270C0E6E2327EC0EF0AD
:1009C000EF500A0803E1010E6F6F02D06C2BE9D7DC
:1009D0006F5101E1FE0C0301DD2B000EDE2327EC3D
:1009E0000EF00B0EDDC3EBFF0C0EDEC3EBFF880E2B
:1009F000D880DD55130EDE5503E2DD6B040EDE6F8D
:100A000027EC0EF027EC0FF0EF9027EC0EF00D0E18
:100A100057C1EBFF0E0E58C1EBFFB5EC0FF01A0EED
:100A200005EC0EF013EC0FF00A0EE66EE66A55C107
:100A3000E6FF56C1E6FF27EC0EF031EC0EF0C1ECFC
:100A40000EF00101020E876F27EC0EF08DEC0FF017
:100A500027EC0EF021EC10F027EC0EF091EC0FF0EB
:100A600027EC0EF095EC0FF027EC0EF06AEC0EF090
:100A700027EC0EF0010EEF6EB5EC0FF0C7EC0EF0A8
:100A80000B016C511200010159511DEC0EF0EF5099
:100A9000030801E0000C010C01015A51240DF3CFB1
:100AA0006CFBF4CF6DFB000E0B016C270C0E6D235D
:100AB0008AEC0EF0EF5003080BE08AEC0EF0EF50DA
:100AC000020806E06CCB91F16DCB92F19AEF0BF03E
:100AD0005AC164F164D9C1EC0EF00101110E876FA7
:100AE0008AEC0EF08DEC0FF08AEC0EF021EC10F099
:100AF0008AEC0EF091EC0FF08AEC0EF095EC0FF012
:100B00008AEC0EF06AEC0EF08AEC0EF0EFEC0FF0CF
:100B100018EC0FF08AEC0EF0040EEF6E12000101DB
:100B20005B51240DF3CF75FBF4CF76FB000E0B0168
:100B300075270C0E762349EC0EF0AEEC0EF001E1B9
:100B4000000C49EC0EF0D5EC0FF0020B01E1000CAB
:100B500049EC0EF0C4EC0FF049EC0EF00F0EEB5028
:100B60000101886F0101180E876F8DEC0FF049ECC1
:100B70000EF021EC10F049EC0EF091EC0FF049EC86
:100B80000EF095EC0FF049EC0EF06AEC0EF049EC2B
:100B90000EF0100E63EC0FF0126A136A49EC0EF0BF
:100BA000EFEC0FF0ECEC0EF049EC0EF027EC0FF050
:100BB000EF9249EC0EF027EC0FF0EF98010C0A0EC3
:100BC00001015C5D01E3000C5C511DEC0EF0140EA4
:100BD00099EC0FF001E1000C5C511DEC0EF00F0ED2
:100BE00005EC0EF0EF50FF0804E10201866B93EF75
:100BF0001DF05C511DEC0EF0D5EC0FF0020B01E086
:100C0000010E120001015D51240DF3CF73FBF4CFEF
:100C100074FB000E0B0173270C0E74238FEC0EF087
:100C2000140E99EC0FF001E1000C8FEC0EF0AEEC1D
:100C30000EF018E10201876BAFEC1DF0E66E8FEC51
:100C40000EF00F0E0FEC10F08FEC0EF0AEEC0EF07D
:100C500001E1000C8FEC0EF0F5EC0EF08FEC0EF0D5
:100C6000CEEC0EF08FEC0EF027EC0FF0EF885EC1AB
:100C700088F2CBEC1DF08FEC0EF0140E05EC0EF0AC
:100C8000EE06EF5A8FEC0EF0100E05EC0EF0EE2A89
:100C9000ED22EECF10F0EDCF11F0CA0E105C030E76
:100CA000115803E35DC15BF13ADF010C01015F51B3
:100CB000240DF3CF6CFBF4CF6DFB000E0B016C2702
:100CC0000C0E6D2353EC0EF0140E99EC0FF001E1B5
:100CD000000C53EC0EF0AEEC0EF018E10201876B45
:100CE000AFEC1DF0E66E53EC0EF00F0E0FEC10F0B3
:100CF00053EC0EF0AEEC0EF001E1000C53EC0EF0F4
:100D0000F5EC0EF053EC0EF0CEEC0EF0FFEC0FF025
:100D100001016251EE24106E6351EE20116ECA0E75
:100D2000D8801054030E11540BE2FFEC0FF0EECFFD
:100D300062F1EFCF63F1CA0ED8806257030E63579A
:100D400053EC0EF027EC0FF0EF8862C18BF263C119
:100D50008CF260C189F261C18AF2E9EC1DF053ECBA
:100D60000EF0140E05EC0EF001016251EE5E6351BF
:100D7000ED5AFFEC0FF06251EE266351ED2253EC79
:100D80000EF0100E63EC0FF0CA0E105C030E11583B
:100D900003E35FC15BF1C3DE010162511200010197
:100DA0006451240DF3CF00FBF4CF01FB000E0B01C7
:100DB00000270C0E012300CBE9FF01CBEAFF1BEC5F
:100DC00010F001E1000C6CEC1FF000CBE9FF01CB4F
:100DD000EAFF1EEC10F0010C01016551240DF3CF68
:100DE00000FBF4CF01FB000E0B0100270C0E0123CA
:100DF000A4EC0EF01BEC10F03CE0A4EC0EF0D5ECF3
:100E00000FF0040B0CE001019C6B9D6B65C19BF125
:100E1000B2EC0DF0A4EC0EF027EC0FF0EF94A4EC84
:100E20000EF0120E63EC0FF001016851105C695175
:100E3000115808E2A4EC0EF015EC10F0EECF68F1BA
:100E4000EDCF69F1A4EC0EF0120E99EC0FF007E172
:100E50006CEC1FF0A4EC0EF01EEC10F00AD068C190
:100E60008FF269C190F266C18DF267C18EF2A1EF77
:100E70001EF0F36AF46A120001016A51240DF3CFE7
:100E800087FBF4CF88FB000E0B0187270C0E88230D
:100E9000896B8A6B8B6BA9EC0EF01BEC10F049E0B0
:100EA000A9EC0EF0D5EC0FF0040B0CE001019C6BEB
:100EB0009D6B6AC19BF1B2EC0DF0A9EC0EF027EC32
:100EC0000FF0EF94A9EC0EF0120E63EC0FF001019D
:100ED0006D51105C000E115809E2A9EC0EF015ECF2
:100EE00010F0EFCF6DF10B01100E896FA9EC0EF031
:100EF000120E99EC0FF009E16CEC1FF0A9EC0EF06A
:100F00001EEC10F0F36AF46A12006EC194F26DC127
:100F100093F26BC191F26CC192F2EDEC1EF0F3CF43
:100F20008AFBF4CF8BFB200E0B01F45C04E1200E56
:100F300001D0300E896F89CB8BFB8ACBF3FF89CB35
:100F4000F4FF120001016F51240DF3CF87FBF4CFA2
:100F500088FB000E0B0187270C0E8823BCEC0EF0DB
:100F60001BEC10F02DE0BCEC0EF0D5EC0FF0040BF8
:100F70000CE001019C6B9D6B6FC19BF1B2EC0DF01D
:100F8000BCEC0EF027EC0FF0EF94BCEC0EF0120E60
:100F900099EC0FF007E16CEC1FF0BCEC0EF01EECCE
:100FA00010F0000CBCEC0EF015EC10F0EE06EF5A51
:100FB00067EC1EF070C1E9FF71C1EAFFEF6E010C32
:100FC000000C0A0E0101725D01E3000C72511DEC70
:100FD0000EF01BEC10F001E0010E12000B017B6B18
:100FE0006C6B0A0E6C5D01E313D16C51240DF3CFD1
:100FF00075FBF4CF76FB000E75270C0E76230EECF6
:101000000EF01BEC10F001E000D10EEC0EF0D5EC70
:101010000FF0100B01E0F9D00EEC0EF0EF500A08C3
:1010200001E1F3D00EEC0EF0EF50000907E10EECF9
:101030000EF0D5EC0FF0010B01E0E7D00EEC0EF056
:101040001F0E05EC0EF00301EE50CC5D106EEE505D
:10105000CD59116E0EEC0EF0210E05EC0EF0FBECEE
:101060000EF01050125C1150135801E3CED0020163
:10107000010E866F93EC1DF0000901E112000EECE9
:101080000EF0C7EC0EF00EEC0EF0210E05EC0EF09B
:10109000010ED890EE36ED36E806FBE10EEC0EF0D0
:1010A0001E0E05EC0EF0EF2A0EEC0EF0EF50090AC2
:1010B00062E0010A58E00F0A65E0020A63E0030AF1
:1010C00061E0020A4AE0070A1FE0010A05E0030A9C
:1010D0005EE10B01020E54D0A0EC0FF003E30B0114
:1010E000120E4ED00EEC0EF0D5EC0FF0010B04E01A
:1010F0000EEC0EF0EF6A46D00B01020E7B6F0EEC89
:101100000EF0010EEF6E3ED0A0EC0FF012E30EECED
:101110000EF0AEEC0EF00AE00201A86BA96B0EEC2B
:101120000EF0CEEC0EF0B9EC20F031D00B01100E29
:1011300027D00EEC0EF0AEEC0EF008E00EEC0EF048
:101140007FEC0EF00EEC0EF09CEC0FF00B01110E8C
:101150007B6F0EEC0EF0040E0CD0A0EC0FF012E33F
:101160000B01010E0DD00B01010E7B6F0EEC0EF08A
:10117000090EEF6E0CD0A0EC0FF004E30B01110E82
:101180007B6F05D075CB91F176CB92F1D3DA0B0161
:101190007B513BE07BA90DD00EEC0EF0EFEC0FF095
:1011A000EECF77FBEECF78FBEECF79FBEFCF7AFB7C
:1011B00010D00EEC0EF0EFEC0FF0EFCF77FBEE2A35
:1011C000EFCF78FBEE22EFCF79FBEE22EFCF7AFB69
:1011D000EF22C1EC0EF07BCB87F10EEC0EF08DEC24
:1011E0000FF077CB7FF178CB80F179CB81F17ACB9F
:1011F00082F10EEC0EF091EC0FF00EEC0EF095EC8F
:101200000FF00EEC0EF06AEC0EF00B016C2BE9D631
:10121000120073C1E9FF74C1EAFF060E05EC0EF07F
:10122000EECF80FBEECF81FBEECF82FBEFCF83FBD7
:1012300075C1E9FF76C1EAFFEECF84FBEECF85FBF7
:10124000EECF86FBEFCF87FB0B01886B060E896F15
:1012500077C18AFB78C18BFB77C1ABF278C1ACF266
:101260001FEC30F0F3CF8AFBF4CF8BFB0C0E0201A6
:10127000B36FB46B0201800EB16F0B0EB26F53EC03
:1012800030F0F3CF8DFBF4CF8EFB0B018D1F8E1F43
:1012900077C1B5F278C1B6F2BFEC30F0F3CF8FFB77
:1012A000F4CF90FB0B01F4508D5D58E18F518E5DB2
:1012B00055E10301706B716B49EC40F0140E0201B3
:1012C0008F6F906B02016C0E8D6F0B0E8E6FA1EC09
:1012D0001EF001016C0E8F6F0B0E906FE8D9D4ECED
:1012E0000EF0106E116A140E105E000E115A10C02E
:1012F00091FB1050106E116AE8500101775D776F15
:1013000011507859786F140E775F000E785BD4EC2B
:101310000EF00301706F716B49EC40F073C18DF1F9
:1013200074C18EF101016C0E8B6F0B0E8C6F42D964
:101330000B018C6FFE0E8C5D11E077C198F178C1C6
:1013400099F101016C0E966F0B0E976F73C194F1BA
:1013500074C195F18CCB93F11DDA010C6CEC1FF08C
:10136000010C0201010E866F93EC1DF0000902E1F1
:101370000400F7D7FF0E0101885D07E10201010EAD
:10138000876FAFEC1DF00101886FFF0E0101885DD2
:1013900001E10FD1140E0201A86FA96B88C1A7F259
:1013A0002FEC21F07BC148FB7CC149FB7DC14AFB8E
:1013B0007EC14BFB7FC14CFB80C14DFB81C14EFB0D
:1013C00082C14FFB83C150FB84C151FB85C152FBDD
:1013D00086C153FB0B01559D559F0B0154915493AE
:1013E0005495549787C155FB7FEC1FF0F3CF56FB04
:1013F000F4CF57FB0B01000E565D040E575905E361
:101400000B01566B040E576F11D00B01360ED880AE
:101410005655000E575507E2360E0B01565F000E6B
:101420000B01575B03D00B01566B576B0B01586BCD
:10143000596B0B015A6B5B6B0101480E8F6F0B0EE2
:10144000906F35D9140E01018927000E01018A23FE
:10145000010187A317D0040E01018927000E0101A5
:101460008A230B01020E5C6F0B01040E5D6F0B01F2
:10147000040E5E6F0B015F6B0B015499548B548DFE
:10148000549F05D00B015489549B548D549FD1C057
:1014900060FBD2C061FBD3C062FBD4C063FB79C1E7
:1014A000E9FF7AC1EAFF060EE926000EEA22EECF36
:1014B00064FBEECF65FBEECF66FBEFCF67FB0B0166
:1014C000686B0B01060E696F89C16AFB8AC16BFBF1
:1014D0006ACBABF26BCBACF21FEC30F0F3CF6AFB14
:1014E000F4CF6BFB0C0E0201B36FB46B0201600E04
:1014F000B16F0B0EB26F53EC30F0F3CF58FBF4CF5B
:1015000059FB0B01581F591F58CB46FB59CB47FBC2
:1015100089C16EF38AC16FF30301060E6D6F79C145
:101520006BF37AC16CF3DAEC3FF0140E02018B6FAF
:101530008C6B0201480E896F0B0E8A6FE9EC1DF06F
:10154000010187A30BD0040E02018B6F8C6B02018B
:101550005C0E896F0B0E8A6FE9EC1DF0140E020110
:10156000A86FA96B88C1A7F22FEC21F089C1B5F251
:101570008AC1B6F2BFEC30F0F3CF46FBF4CF47FBA5
:10158000240E0201A86FA96B88C1A7F22FEC21F0ED
:1015900047CB88F2CBEC1DF046CB88F2CBEC1DF0AC
:1015A0000201A86BA96B88C1A7F22FEC21F0B9EC5E
:1015B00020F012000B01FE0E036F026B0A0E025D9B
:1015C00051E20251DEEC0EF073DBEF500A0847E007
:1015D0006FDB0B0E63EC0FF01DEC0FF0020E15DB52
:1015E000FBEC0EF000011250101839E113501118E5
:1015F00036E15EDBEF50000902E102CB03FB58DB72
:101600000D0E63EC0FF01DEC0FF0FBEC0EF0125022
:10161000101825E11350111822E18DC1E9FF8EC188
:10162000EAFF060EF2DAEECF14F0EECF15F0EECFB1
:1016300016F0EFCF17F03CDBEE52060E18EC10F070
:1016400014180DE1EE5015180AE1EE50161807E1D6
:10165000EE50171804E103E10B01025112000B01D7
:10166000022BACD7FE0E035D01E1FE0C0351A6DB9D
:101670000A0EE66EE66A8DC1E6FF8EC1E6FF18DB54
:10168000F0DA1250DADB0ADB13DBBADB11DB1EEC1B
:1016900010F00EDB63DB05E00BDB31DB09DB9CECE0
:1016A0000FF006DBD4DBEF820B0103511200C0DA2E
:1016B000EFCF07FB06EC10F08BDBBADA74EC0FF01F
:1016C000020E85EC0FF0020EE6DB020E8AEC0FF044
:1016D000020E12EC10F0040EE1DB040EBAEC0FF077
:1016E000080EDCDB080EBAEC0FF00E0E85EC0FF0E6
:1016F0000E0ED1DB0E0E8AEC0FF00E0E12EC10F077
:10170000100E85EC0FF0100EC6DB100E8AEC0FF0F9
:10171000100E12EC10F0120E85EC0FF0120EBBDB67
:10172000120E8AEC0FF015EC10F0010E6EDA07CBFA
:10173000EFFF120091DA12DB08E08EDAE0DA8CDAE1
:101740009CEC0FF089DA83DBEF8286DACBEC0FF0CA
:1017500083DA0D0EEB6A0E0EEB6A7EDA1BEC10F0EC
:1017600002E06CEC1FF078DA1EEC10F075DAC0ECD9
:101770000FF072DA6CDBEF986FDAD5EC0FF0010B3B
:1017800003E06ADAEF6A03D067DA0A0EEF6E64DA12
:10179000D0EF0FF001019351240DF3CFA2FBF4CF52
:1017A000A3FB000E0B01A2270C0EA32398C151F13D
:1017B00099C152F1A46B2DDA1E0E27DAEF6A29DAED
:1017C000E6DA27DADDDB3EDB040B0DE06CEC1FF024
:1017D00020DAEBDB010B02E0000E01D0010EE66E19
:1017E00018DAE8EF0EF054DBB0DB0E0E0EDAEECFB7
:1017F00014F0EFCF15F0166A176A15DA080E18EC18
:1018000010F0965D186EEE509759196EEE5098597B
:101810001A6EEE5099591B6E1850145C106E1950C8
:101820001558116E1A501658126E1B501758136E19
:10183000F0D9100EEAD9EECF1CF0EFCF1DF01E6AE2
:101840001F6A1C50105C926F1D501158936F1E50F0
:101850001258946F1F501358956F800E951506E01F
:10186000D8D9140EEB6A150EEB6A07D0D2D9140E34
:1018700092CBEBFF150E93CBEBFFC5DB01081EE10E
:10188000E1DA020B05E1A4DB100B01E15AD11CD017
:10189000E1DA8EDB49DADBDB06E1BBD9020EEF6E63
:1018A0006CEC1FF02AD0B5D9030EEF6E100EA46FAA
:1018B00099DB01019851991166E1B9D0A4DB0009C7
:1018C00020E186DB020B03E10B01040E18D0C2DA23
:1018D00089DB0A0EE66EE66A94C1E6FF95C1E6FF73
:1018E00098D9BFD912509FD9D9D993D989DA91D92A
:1018F000020EEF6ECDDAEADA17DA0B01120EA46FE0
:10190000D3D056DBEECF9AFBEECF9BFBEECF9CFB0A
:10191000EFCF9DFBBDDAEECF9EFBEECF9FFBEECF70
:10192000A0FBEFCFA1FB7FD9040E6FD9FDD9010138
:1019300098510B019227010199510B019323000E3D
:1019400094239523A5DA01DB040E72DB9A1901E0DA
:101950009ED0EE509B1901E09AD0EE509C1901E008
:1019600096D0EE509D1901E092D001E090D04BDB73
:1019700002080BE16CDB5BE0BDDA030EEF6E0101E8
:101980009851991154E018DB8FD0B4DAEF50030866
:1019900051E15DDB23E047D9080E37D9EECF10F0D7
:1019A000EECF11F028DA74DA1050EE1817E111506A
:1019B000EE1814E11250EE1811E11350EE180EE17A
:1019C0000DE127D9F2DA020B09E123D9C7D906E0E4
:1019D00020D995D91ED9B0DA37DBEF8233DA010B83
:1019E00009E00B01110EA46F53DA70DA66D911D930
:1019F000090EEF6E01019851991119E00AD91BDB0C
:101A000004E1DADA0B01A4894FD042DA9ECBEEFF73
:101A10009FCBEEFFA0CBEEFFA1CBEEFFC9DA9ACBB6
:101A2000EEFF9BCBEEFF9CCBEEFF9DCBEEFF6CEC75
:101A30001FF03AD0E8DA090804E1CADA100B34E002
:101A400020D0E1DA04080FE1C3DA010B06E087DAFF
:101A5000FEDA17E1DED8060E04D0F9DA25E0D9D88F
:101A6000050EEF6E21D0CFDA050805E1B1DA010BE2
:101A70001BE075DA06D0C7DA060816E1A9DA100B02
:101A800013E0A2CB91F1A3CB92F154DE0DD06CEC1C
:101A90001FF00B01100EA46F9ACB92FB9BCB93FB14
:101AA0009CCB94FB9DCB95FB0B01A4514AE0B1D894
:101AB0007CDA020B28E1ADD851D925E0AAD8100E66
:101AC00038DA21E095DA1050EE5E1150EE5A1250DD
:101AD000EE5A1350EE5A9DD857DA9BD80F0EEB50A2
:101AE0000101886F080E0B01A4110101876F15DA3F
:101AF000CFD9FCD88ED815DA8CD817DA8AD8EAD89C
:101B000077DAECEF0EF03DD9A4CB87F192CB83F1DD
:101B100093CB84F194CB85F195CB86F196CB7FF175
:101B200097CB80F198CB81F199CB82F17CD81AD9EF
:101B30007AD8020E6AD81BD994C179F195C17AF18D
:101B400010DC120001019A51240DF3CF10F0F4CFF4
:101B500011F0000E10260C0E112210C0F3FF11C060
:101B6000F4FF120001019B51240DF3CF8DFBF4CF44
:101B70008EFB000E0B018D270C0E8E230C0E030125
:101B8000706F716B49EC40F067EC1EF0E840E84084
:101B90003F0B3C0B0B018C6F01019C51515D106E92
:101BA00052519D55116E8DCBE9FF8ECBEAFF120E7F
:101BB00010C0EBFF130E11C0EBFF0B018C510101A4
:101BC0009C250301706F000E01019D210301716FBF
:101BD00049EF40F001019E51240DF3CF00FBF4CFFB
:101BE00001FB000E0B0100270C0E012300CBE9FFC7
:101BF00001CBEAFF1ADA0101EE50515D106EEE5092
:101C0000525910C0F3FFF46E1200E926000EEA22CA
:101C10001200A2CBE9FFA3CBEAFF120075CBE9FFCC
:101C200076CBEAFF120096C1E9FF97C1EAFF1200E6
:101C30008FC1E9FF90C1EAFF1200240DF3CFE9FF45
:101C4000F4CFEAFF000EE9260C0EEA2212006DCB5B
:101C5000E9FF6ECBEAFF120091C1E9FF92C1EAFFF2
:101C60001200EE52E9CF10F0EACF11F0E9CFE6FF13
:101C7000EACFE6FF66EC47F0126E060EE15E120058
:101C8000EECF83F1EECF84F1EECF85F1EFCF86F189
:101C9000120075CBE9FF76CBEAFF1200EECF10F011
:101CA000EFCF11F012006CCBE9FF6DCBEAFF120011
:101CB00000CBE9FF01CBEAFF1200EF2AEECF92FB47
:101CC000EF22EECF93FBEF22EECF94FBEF22EFCF8C
:101CD00095FB1200EE52E9CF79F1EACF7AF1B1EF3C
:101CE00009F001CBE9FF02CBEAFF1200EECF7FF152
:101CF000EECF80F1EECF81F1EFCF82F112000F0E27
:101D0000EB500201966F62EF1FF001CBE9FF02CBAF
:101D1000EAFF12006CCBE9FF6DCBEAFF120073CB38
:101D2000E9FF74CBEAFF1200EECF92FBEECF93FBFC
:101D3000EECF94FBEFCF95FB120011C0EEFF12C067
:101D4000EEFF13C0EEFF120000CBE9FF01CBEAFF6C
:101D5000120087CBE9FF88CBEAFF12000F0EEB5091
:101D6000FF081200EECF7DF1EDCF7EF11200EECF35
:101D70007BF1EDCF7CF1120087CBE9FF88CBEAFF46
:101D800012000101896B8A6B0101886912001F0E24
:101D9000CCC3EBFF200ECDC3EBFF12000F0EEB50B8
:101DA0000201A76F2FEF21F00B017851F00BE842F1
:101DB000E842E842E842040DF3501200240DF3CF4C
:101DC00000FBF4CF01FB000E00270C0E01231200D4
:101DD000E552E750EF6E12001050EE261150EE2241
:101DE0001250EE221350EE221200DAD8280E020111
:101DF000A86FA96B1200EECF12F0EFCF13F0120014
:101E00000D0E10C0EBFF0E0E11C0EBFF1200140EF2
:101E100010C0EBFF150E11C0EBFF12002C0EEE6E82
:101E2000010EED6E1200EE6AEE6AEE6AEE6A1200C4
:101E3000EE2AEE22EE22EE2212008BC1E9FF8CC1C7
:101E4000EAFF1200F0DE0D0EE0DEEF501200230E6E
:101E500005EF0EF098C114F099C115F0166A176AD3
:101E6000E2DE040EE5D81424106EEE501520116E3B
:101E7000EE501620126EEE501720136E102A000E30
:101E800011221222132294D810C0EEFF9DEF0EF003
:101E9000C0DEEFEF0FF0B9DE06EF10F0B6DEEECFEA
:101EA000ADF2EECFAEF2EECFAFF2EFCFB0F224EC68
:101EB00030F004C010F005C011F006C012F007C0E9
:101EC00013F018EF0EF0A1DE4EEF0EF0EFCF96FB01
:101ED000EE2AEFCF97FBEE22EFCF98FBEE22EFCF6B
:101EE00099FBEF22D8EF0FF0010E8FDE07CBEFFF4B
:101EF00018EF0EF05DD892CBEEFF93CBEEFF94CBB4
:101F0000EEFF95CBEEFF09EF0EF07FDEEFCF07FB84
:101F100018EF0EF084D818EF0EF01A0E76DE40EFB0
:101F20000EF00D0E72DEB2EF0EF00B0E6EDEB7EF9E
:101F30000EF07ED8ED1012000F0E67DEEF68120073
:101F40006DDE1E0EEB5003081200EECF96FBEECFB7
:101F500097FBEECF98FBEFCF99FB13EF0EF00B0141
:101F6000100EA46F25D85DEF0EF071DE38D860DF5B
:101F700027EF0EF04ADE04C0EEFFDFDE18EF0EF0B2
:101F8000210E43DE0EEF0FF0100E3FDEEECF89F193
:101F9000EDCF8AF11200EE52060E37DE13EF0FF08E
:101FA000100EEB6A110EEB6A120051DFEF501200B7
:101FB00030DE1A0E05EF0EF047D8EF862ADE120E3D
:101FC00098C1EBFF130E99C1EBFF3ED8EF841200CE
:101FD0006CEC1FF022EF0FF098DE27EF0FF0160EDB
:101FE00005EF0EF020DE0E0E6EDF13DE07EF0FF0B2
:101FF00010DE100E68DF126A136A48EF0FF053DE2E
:10200000100E05EF0EF005DEEF501200010EFDDDA3
:10201000EF50E66E18EF0EF064DE27EF0FF0F5DDFF
:10202000E8EF0EF0F2DD74EF0FF0120E05EF0EF098
:10203000ECDDEE501200B9DF080B120008DFEF965E
:102040001200CDDF76EF0EF0E4DD27EF0FF0FADEC1
:04205000100B12005F
:0C205400CCC33CFFCDC33DFF0B01036B70
:10206000060E035D2FE20001750EEF6FFEEC37F0F8
:10207000116E106A10C0E6FFE66E0001740EEF6F7D
:10208000FEEC37F0E552E7CF11F0E552E7CF10F064
:1020900001011010536F11C054F189EC04F0E66E89
:1020A0000B0107EC16F0E552E750EF6E07EC16F067
:1020B00005EC16F0EF6A07EC16F0DCEC15F0EF6AB1
:1020C000032BCED712000B01CC6B060ECC5D06E2C3
:1020D000CCCB43FF8ED80B01CC2BF7D712003ECFD1
:1020E00000FB3FCF01FB0B0100CBE9FF01CBEAFF77
:1020F000002B000E0123EF502E0807E000CBE9FF74
:1021000001CBEAFFEF50EFE10A0C026B0251106EB7
:10211000116A100E105C000E115815E20251DEEC2F
:1021200015F000CBE6FF01CBE6FFB1EC47F0136EF4
:10213000050EE15E1350000903E10B01025112008C
:102140000B01022BE3D70A0C1CEC16F004E0200E66
:102150000B01005DF9E00B01016B2B0E0B01005D23
:1021600002E1200E006F2F0E005D20E05C0E005D8E
:102170001DE0200E005D1DE03F0E005D1AE00D0E1B
:10218000005D17E00A0E005D14E00C0E015D0EE22A
:10219000610E005D05E300517A0802E3200E005F46
:1021A0000151012B33EC16F000CBEFFF1CEC16F0C5
:1021B000D4E10B01015133EC16F0EF6A0B01015130
:1021C00012E1CD0E106E930E116E126A10C0E6FF72
:1021D000E66E12C0E6FF41CFE6FF42CFE6FFC7EC56
:1021E00047F0050EE15E3F0E0B01005D01E1010CC1
:1021F000000C0F0143510A0DF3CFC5FBF4CFC6FB12
:10220000000E0B01C5270F0EC623010EC36F0B0175
:10221000C35101E1F8D1C36BCB6BD3EC15F03AECB1
:1022200016F00DE19AEC16F0020B02E095EC16F0B8
:1022300052EC16F0EF9458EC16F0EF6A1200D3EC63
:1022400015F0020EEB50080AE2E00F0A01E1CBD1D3
:10225000010A01E19CD1030A01E199D1010AD7E009
:10226000070A01E1BCD1010A01E171D1030A01E1D0
:102270002DD1010ACCE1D3EC15F047EC16F0C7E004
:102280000B01010EC36FCCC33CFFCDC33DFF52EC2D
:1022900016F0EF6A7FEC16F00F01496F11DA0B01AF
:1022A000C26F0F01B50E416F0B0E426F7FEC16F03F
:1022B0000F01406F49DF0B01CB91E8B0CB817FEC80
:1022C00016F001019E6FEAEC0DF0F3CFC9FBF4CFDD
:1022D000CAFB0F01B50E506F0B0E516F43CF4FFF6E
:1022E00069EC15F00F01B50E3E6F0B0E3F6FF7DE78
:1022F0008EEC16F0060814E055EC16F0EF0402E040
:10230000000E01D0010E000E00090AE1A1EC16F04A
:10231000040802E0000E01D0010E000E000904E0E6
:1023200052EC16F0EF8003D052EC16F0EF9000EC78
:1023300016F0020B22E1A1EC16F0060804E100EC15
:1023400016F0100B1AE1580E0B01B55D04E100EC1C
:1023500016F0010B12E19AEC16F0010B04E000EC10
:1023600016F0080B0AE100EC16F0040B0DE00B016F
:10237000C2510AE1CB51010B07E09AEC16F0040BB5
:1023800003E182EC16F03DD00B01C25101E098D080
:1023900052EC16F0CB93EF50040B01E0CB8300EC32
:1023A00016F0200B03E152EC16F0EF840B01CBA1E9
:1023B00015D0C9CB9CF1CACB9DF17FEC16F0010181
:1023C0009B6FB2EC0DF00201B50EE66F0B0EE76FDE
:1023D000C5CBE4F2C6CBE5F2A9EC29F052EC16F03D
:1023E0000B01CB51020B02E0EF8401D0EF9482ECA1
:1023F00016F09AEC16F0100B0DE09AEC16F0040BA8
:1024000009E16BEC16F0020EEF6ECDDB9DEC16F0E1
:10241000060EE7D058EC16F0050EEF6E5BEC16F0EA
:1024200085EC16F0106E060E105C2FE3A1EC16F092
:1024300004082BE3B50EE66E0B0EE66EE0EC47F0FB
:10244000E552E552F3CFC4FBA1EC16F0030802E31A
:10245000030E01D0020E0B01C45FA1EC16F00B0FAE
:102460008EEC16F0ABDBC451146AB50F136E0B0E75
:10247000142213C0E6FF14C0E6FFC7EC47F0156E48
:10248000050EE15E15505BEC16F085EC16F0FF08CA
:1024900004E16BEC16F0EF6A08D085EC16F0FE084C
:1024A00008E16BEC16F0010EEF6E58EC16F0050E1D
:1024B00098D052EC16F0EF8258EC16F0010E91D045
:1024C000C20501E0A4D6F4DB030E8BD089EC16F034
:1024D00001E19DD60B01010EC36F0F01560E4D6F2A
:1024E000930EA0DBDBDB0F01660E4D6F930E9ADBC4
:1024F000DCDBEF34EA6AFE0BEA36E96E000EE92611
:10250000030EEA22EECF4DFFEDCF4EFF43CF4CFF3F
:10251000BBDAC4DBCADBEFCF10F00B0E105C05E3B7
:102520000F01750E4D6F930E7DDB9AEC16F0010BCB
:1025300005E10F01BC0E4D6F770E74DBAFDB33DBB3
:10254000030E9DEC16F0EF6AB3DB020E4AD02BDBD4
:102550009EDB01E0D7DBA6DB0B01CB93EF50040B36
:1025600001E0CB834DDB200B02E19CDBEF8443CF0A
:102570004AFFE9D8000904E0D8DB9ADB070EEF6ECA
:1025800091DB0B01CB51020B3CE0EF8440D6C1DB69
:1025900001E13DD6A0DBEF34EA6AFE0BEA36E96ED4
:1025A000200EE926030EEA22EECFC7FBEDCFC8FBD3
:1025B0000B01C7CBF6FFC8CBF7FFC72B000EC82314
:1025C0000800F5CFC4FBF55005E0C4CB5EF1EBDAB3
:1025D0002EDBEED794DB01015B6F8FEC05F068DB3F
:1025E000070EEF6E14D6DFDA45DB0AE092DB08E077
:1025F00086DB01015A6F4CEC05F05ADB080EEF6EDA
:1026000051DBEF9404D6120047CFE9FF48CFEAFF31
:10261000EF040B014A6F496BEF6A4B6B4A510F0194
:10262000EA6A4525E96E4651EA22EF6A0B014B51F1
:1026300041E10101480E706F0B0E716F44CF6FF1D5
:10264000A2EC07F0000936E03D0E0B01485D0BE1FE
:10265000486B4A51495D1EE2492947CFE9FF48CFFF
:10266000EAFFEF6E17D0260E485D02E1020E0AD097
:10267000200E485D06E00D0E485D03E00A0E485D41
:1026800004E1010E4B6F486B05D02B0E485D02E153
:10269000200E486F4A51495D06E245CFE9FF46CF1B
:1026A000EAFF48CBEFFF0F01452B000E46230B013D
:1026B000492BBCD70B014B5101E1000C4B0512001B
:1026C0000B01056B0101060E706F0B0E716F49CF88
:1026D0006FF1A2EC07F0000916E0200E0B01065D79
:1026E00012E00551106E116A040E105C000E1158B4
:1026F000E9E20551052BEA6A000FE96E0B0EEA22AA
:1027000006CBEFFFDFD70B010551EA6A000FE96E38
:102710000B0EEA22EF6A470E005D07E1450E015DF0
:1027200004E1540E025D01E1000C500E005D0AE16F
:102730004F0E015D07E1530E025D04E1540E035D8F
:1027400001E1010C020C0F014A510A0DF3CF6EFB9F
:10275000F4CF6FFB000E0B016E270F0E0B016F23E2
:102760006ECBE9FF6FCBEAFFEF5001015C6FDFEC4E
:1027700005F0000901E168D10B016C6B6ECBE9FF3C
:102780006FCBEAFF030EEB50040846E06ECBE9FF87
:102790006FCBEAFF010EEB50080DF3CFE9FFF4CF4A
:1027A000EAFF000EE926020EEA22EF50400B0BE092
:1027B0006ECBE9FF6FCBEAFFEF5001015B6F8FEC4F
:1027C00005F0010E4DD16ECBE9FF6FCBEAFF010E94
:1027D000EB500201386FC4EC36F00B016D6F6ECB1D
:1027E000E9FF6FCBEAFF010EEB50080DF3CFE9FFD5
:1027F000F4CFEAFF000EE926020EEA22EF50200B8A
:102800000BE06ECBE9FF6FCBEAFFEF5001015B6F8E
:102810008FEC05F0010E24D16ECBE9FF6FCBEAFF00
:10282000090EE926000EEA22EF50010B01E1FFD06C
:102830006ECBE9FF6FCBEAFF030EEB50040A01E118
:10284000ABD0070A73E0010A42E0030A16E0010A6E
:1028500001E0DDD0250E0B016D5D0BE16ECBE9FFD4
:102860006FCBEAFF030EE926000EEA22010EEF6E9F
:1028700003D00B01010E6C6FCBD0250E0B016D5DEB
:102880000DE10B01010E6C6F6ECBE9FF6FCBEAFF20
:10289000030EE926000EEA22EF6A18D06ECBE9FF9C
:1028A0006FCBEAFF040EE926000EEA22030EE926AA
:1028B000000EEA226DCBEFFF6ECBE9FF6FCBEAFF94
:1028C000030EE926000EEA22020EEF6EA1D0610E81
:1028D0000B016D5D04E3270E0B016D5F07D0410E08
:1028E0000B016D5D03E3070E0B016D5F300E0B01F5
:1028F0006D5D100DF350E66E6ECBE9FF6FCBEAFF16
:10290000040EE926000EEA22020EE926000EEA2253
:10291000E552E750EF6E6ECBE9FF6FCBEAFF030E97
:10292000E926000EEA22030EEF6E72D0610E0B0153
:102930006D5D04E3270E0B016D5F07D0410E0B01A7
:102940006D5D03E3070E0B016D5F300E0B016D5DD6
:10295000106E6ECBE9FF6FCBEAFF040EE926000E86
:10296000EA22020EE926000EEA221050EF126ECB88
:10297000E9FF6FCBEAFF030EE926000EEA22040E00
:10298000EF6E6ECBE9FF6FCBEAFF040EE926000E77
:10299000EA22EE6AED6A3CD002016D0EEA6F0B0E80
:1029A000EB6F6ECBE8F26FCBE9F221EC2AF0F3CFBC
:1029B00010F0F4CF11F06ECBE9FF6FCBEAFF040EFD
:1029C000E926000EEA2210C0EEFF11C0EDFF0B0158
:1029D000010E6C6F6ECBE9FF6FCBEAFF040EE926A8
:1029E000000EEA22FF0EEE1802E1FF0EED180EE1D6
:1029F0000B016D5102E10B016C6B6ECBE9FF6FCBEC
:102A0000EAFF030EE926000EEA22EF6A01D000D0A9
:102A10000B016C510BE06DCB5EF16ECBE9FF6FCB20
:102A2000EAFFEF5001015D6F02EC06F00BD06DCBB9
:102A30005EF16ECBE9FF6FCBEAFFEF5001015D6FF6
:102A400002EC06F004008CD66ECBE9FF6FCBEAFFF8
:102A5000010EEB500201376F90EC36F0000E00D003
:102A600012000F014B510A0DF3CF6CFBF4CF6DFB3D
:102A7000000E0B016C270F0E6D2301010D0E38D9CE
:102A800001010A0E78EF16F00F014C510A0DF3CF39
:102A90006CFBF4CF6DFB000E0B016C270F0E6D234A
:102AA0004DCFF6FF4ECFF7FF0800F55011E00F01B4
:102AB0004DCFF6FF4ECFF7FF4D2B000E4E230800F3
:102AC000F5CF5EF16CCBE9FF6DCBEAFFB0D8E8D76C
:102AD00012000F014F510A0DF3CF00FBF4CF01FBA1
:102AE000000E0B0100270F0E0123040E836F01015E
:102AF0000A0E79D801E1115006E00B0183518307DA
:102B00000009F5E1120001010D0E6E6F0101800E4A
:102B10006D6F0101020E6B6F0B0E6C6FE0D8F3CF7F
:102B200085FBF4CF86FB0B01F45010E1040E836F9C
:102B300001010D0E58D801E1115005E00B01835140
:102B400083070009F5E10B01200E866F200E865DDC
:102B500001E01200850501E112000101830E706F92
:102B60000B0E716F00CBE9FF01CBEAFFEF500101C3
:102B70006F6FA2EC07F00B018505EA6A020FE96EA0
:102B80000B0EEA22EF6A50CFA9F351CFAAF303014B
:102B9000020EA76F0B0EA86F00CBA5F301CBA6F317
:102BA0009DEC3EF0B0D7C5CBE9FFC6CBEAFF1200E3
:102BB000040EC3D8040EB0D0090EAED0040DF3CF6E
:102BC000F6FFF4CFF7FF160EF626930EF722F6CF98
:102BD00010F0F7CF11F0126A10C0E6FF11C0E6FF47
:102BE00012C0E6FF12006E6F01016D6901016B6B8F
:102BF0006C6B75D8F4CF10F0116A200EF418120027
:102C00000001720EEF6FFEEF37F0020E85D0035118
:102C10000A0DF3CFE9FFF4CFEAFF000EE9260F0E0D
:102C2000EA2212004E6F43CF4CFF44EF15F0EF50F5
:102C300001015D6F02EF06F00101000E706F0B0ED7
:102C4000716F40CF6FF1A2EC07F000091200EF5056
:102C500001015C6FDFEC05F000091200EF5001018B
:102C6000646FCFEF06F00F01EA6A4125E96E425129
:102C7000EA221200EF500101596F43EC05F0000900
:102C80001200010EEB500201366F88EF36F0EF5064
:102C90000101726FE1EC07F00009120043CF4BFF16
:102CA00031EF15F080DFDCEF15F07DDFD8EF15F0A8
:102CB0007ADF05EF16F00201356B0201B50E336FB6
:102CC0000B0E346F80EC35F0E66E6DDFEE52E552A0
:102CD000E750EF6E120067DF040E9DEF16F000CB99
:102CE000E9FF01CBEAFFEF5001016A6F3CEF07F00B
:102CF0005E6F6CCBE9FF6DCBEAFF17EF16F053DF89
:102D0000EF50120050DF2EEF16F04DDF010EEB50AA
:102D1000120049DF27EF16F09DEF16F0E66EC5DFD3
:102D2000E552E750EF6EA1EF16F0BCDFEF923BDF0C
:102D300041EF16F0B7DFEF501200E926000EEA224D
:082D40001200B3DFEF50120096
:082D48000001FA6B0A0E020102
:102D5000D06FD16B0201000ECE6F0B0ECF6F17EC50
:102D600032F00001B56BB66B0001000EB36F0B0EB5
:102D7000B46F00015C0EEF6FFEEC37F0116E106A5D
:102D800010C0E6FFE66E00015B0EEF6FFEEC37F061
:102D9000E552E7CF11F0E552E7CF10F00001101037
:102DA000B16F11C0B2F0EFEC25F00301E16FFF0E3F
:102DB000E15D12000B01476B0001FA5124E1E1C310
:102DC000BEF06FEC27F000093EE00001620EEF6FED
:102DD000FEEC37F0010B2DE00001010EFA6F00014F
:102DE000620EEF6FFEEC37F0020B04E00B01010EF8
:102DF000436F04D00B01010E476F436B006B026BF6
:102E0000466B426BCBD0FA051CE10B0100B117D029
:102E100000A303D00001FA6B16D0006B0001010E75
:102E2000BF6F0B0EC06F7EEC27F0000905E10B01B0
:102E30000083CCEC27F007D00B01009304D0009165
:102E400002D0020EFA5D0001FA5101E1A7D00B0198
:102E50004351070A01E1A1D0010A01E19BD0030A15
:102E600001E196D0010A01E178D0070A5FE0010A8A
:102E700045E0030A0EE0010A01E090D000B38ED0D5
:102E8000250E015D02E1050E86D0020E436F008122
:102E900085D0200E015D28E10251A0EC1CF0EF6A04
:102EA000350E0201C86FC96B0201030EC66F0B0E0F
:102EB000C76FCCEC31F0000913E13E0E0201C86F80
:102EC000C96B0B0146510201C66FC76B030EC627C3
:102ED0000B0EC723CCEC31F0000902E10B01436B70
:102EE0000B01026B466B5AD03A0E015D03E1016B98
:102EF0000229466FA6EC1CF051E228D03D0E015D80
:102F000012E1016B030E436F0229106E116A400E2D
:102F1000105C000E11580AE20229466F0229A0EC4B
:102F20001CF0EF6A03D0200E015D2FE000A304D057
:102F3000040E436F008107D0260E015D04E1040EEC
:102F4000436F0081016BA6EC1CF028E20251022BBA
:102F5000A0EC1CF001CBEFFF21D047CBFFF0465196
:102F60000001FD6FFE6B030EFD270B0EFE2300011B
:102F7000030EFB6F0B0EFC6F16D8F3500B014413BE
:102F8000F450451300B30AD0436B466B026B06D076
:102F9000060E01D0070E436F01D0436B0001FA51BA
:102FA00001E00AD712000B01486B496BFBC0E9FF37
:102FB000FCC0EAFFEF506B0801E02CD10B01010EC1
:102FC0004C6F0201500EBA6F0B0EBB6F010E000169
:102FD000FB250201B86F000E0001FC210201B96F50
:102FE00039EC31F0000904E1F36AF46A9FEF1CF058
:102FF000030E0001EA6AFB25E96EFC51EA22EF505C
:1030000062082AE1040E0001EA6AFB25E96EFC5120
:10301000EA22EF50D00F106E010E105204E0E84685
:10302000FE0B1006FCE10B01526F50CBEFF0FEECF3
:1030300037F00B01516FFDC0E9FFFEC0EAFFEF5012
:10304000300805E10B01521D0B01511704D00B0193
:1030500052510B01511361D0FDC0E9FFFEC0EAFFE0
:10306000EF50480818E10201510EBA6F0B0EBB6F0A
:10307000010E0001FD250201B86F000E0001FE21C6
:103080000201B96F39EC31F0000904E1F36AF46A26
:103090009FEF1CF00AD0FDC0E6FFFEC0E6FF47EC44
:1030A00044F0E552E552F3CF51FB030E0001EA6A0A
:1030B000FB25E96EFC51EA22EF506D082EE102017A
:1030C000520EBA6F0B0EBB6F040E0001FB250201FE
:1030D000B86F000E0001FC210201B96F39EC31F02C
:1030E000000904E1F36AF46A9FEF1CF00B01521D22
:1030F000106E10C0E6FF50CBEFF0FEEC37F0E5525B
:10310000E7CF10F010140B01536F0B0151510B015D
:1031100052150B0153110B01516F0B015051110846
:1031200004E2160E0B01505D05E10B0148830B0113
:103130004C6B63D00B015051150809E3130E0B01C2
:10314000505D04E00B01488F0B014C6B56D00B0116
:1031500050511A0801E351D00B0150511E0801E3F0
:103160004CD00B015051220817E31F0E0B01505D8C
:1031700004E0210E0B01505D07E10B0151510808DD
:1031800002E30B014C6B02D00B014C6B0B014C5159
:1031900002E10B01488531D00B015051300805E3A5
:1031A0000B0148870B014C6B28D00B0150513208A2
:1031B00005E30B0148890B014C6B1FD00B015051EB
:1031C0005A0803E30B014C6B18D00B0150516208F5
:1031D00003E30B014C6B11D00B0150516F0805E359
:1031E0000B0149810B014C6B08D00B015051750844
:1031F00004E30B0149830B014C6B0B014C5109E1BA
:103200000001FF5106E051CBA8FF50CBF0F00BECD2
:1032100038F090D3FBC0E9FFFCC0EAFFEFCF10F01D
:10322000610E105C01E203D2FBC0E9FFFCC0EAFFC3
:10323000EF50670801E2FBD1FBC0E9FFFCC0EAFFE9
:10324000EF50640807E0FBC0E9FFFCC0EAFFEF5065
:10325000650803E1F36AF46A72D3FBC0E9FFFCC0BE
:10326000EAFFEF509F0F0B014A6F4B6B890E0B016A
:103270004A270F0E0B014B23010E0001EA6AFB25C2
:10328000E96EFC51EA22EF5014E102014C0EBA6FD4
:103290000B0EBB6FFDC0B8F2FEC0B9F239EC31F0D5
:1032A000000906E04ACBE9FF4BCBEAFF4CCBEFFF2E
:1032B000BDD1010E0001EA6AFB25E96EFC51EA224C
:1032C000EF50780833E1020E0001EA6AFB25E96E4F
:1032D000FC51EA22EF50D00F106E010E105204E0A4
:1032E000E846FE0B1006FCE10B014F6FFDC0E9FF45
:1032F000FEC0EAFFEF5031080AE10B014F1D106ECE
:103300004ACBE9FF4BCBEAFF1050EF160ED0FDC0C1
:10331000E9FFFEC0EAFFEF50300807E14ACBE9FFC2
:103320004BCBEAFF0B014F51EF1280D1010E000190
:10333000EA6AFB25E96EFC51EA22EF50630801E0DE
:1033400077D0020E0001EA6AFB25E96EFC51EA2201
:10335000EF50D00F0B014F6F0B014F51070867E380
:10336000010E4FCBE7FFE75204E0E846FE0BE7060D
:10337000FCE10B014F6FFBC0E9FFFCC0EAFFEF501F
:103380009F0F0B014A6F4B6B920E0B014A270F0EDA
:103390000B014B23FBC0E9FFFCC0EAFFEF509F0F7E
:1033A000230F0001EF6FFEEC37F00B014E6FFDC0F5
:1033B000E9FFFEC0EAFFEF5031080CE14ACBE9FF1C
:1033C0004BCBEAFF0B014F51EF120B014F510B0199
:1033D0004E1316D0FDC0E9FFFEC0EAFFEF503008E3
:1033E0000FE10B014F1D0B014F6F4ACBE9FF4BCB98
:1033F000EAFF0B014F51EF160B014F510B014E1716
:10340000030E0001EA6AFB25E96EFC51EA22EF5047
:1034100072080DE14ECBA8FFFBC0E9FFFCC0EAFF3C
:10342000EF509F0F230F0001F06F0BEC38F0FED030
:10343000010E0001EA6AFB25E96EFC51EA22EFCF9A
:1034400010F0300E105C01E2F1D0010E0001EA6ACA
:10345000FB25E96EFC51EA22EF50390801E2E6D083
:10346000010E0001EA6AFB25E96EFC51EA22EF50E9
:10347000D00F0B014F6F020E0001EA6AFB25E96EC7
:10348000FC51EA22EF500AE0020E0001EA6AFB2535
:10349000E96EFC51EA22EF50720859E1010E4FCB60
:1034A000E7FFE75204E0E846FE0BE706FCE10B010C
:1034B0004F6FFBC0E9FFFCC0EAFFEF509F0F2A0FE0
:1034C0000001EF6FFEEC37F00B014E6FFDC0E9FF1E
:1034D000FEC0EAFFEF50300810E10B014F1D0B0159
:1034E0004F6F4ACBE9FF4BCBEAFF0B014F51EF1671
:1034F0000B014F510B014E1712D0FDC0E9FFFEC06A
:10350000EAFFEF5031080BE14ACBE9FF4BCBEAFF72
:103510000B014F51EF120B014F510B014E13020ED5
:103520000001EA6AFB25E96EFC51EA22EF507208BD
:103530000DE14ECBA8FFFBC0E9FFFCC0EAFFEF5056
:103540009F0F2A0F0001F06F0BEC38F06FD0020EC6
:103550000001EA6AFB25E96EFC51EA22EF5070088F
:103560000AE0020E0001EA6AFB25E96EFC51EA223C
:10357000EF506E085BE1010E4FCBE7FFE75204E02E
:10358000E846FE0BE706FCE10B014F6FFDC0E9FFCB
:10359000FEC0EAFFEF50D00F0B014C6F000E0B0185
:1035A0004C5D04E30B014C51090802E20B014C6B2A
:1035B000020E0001EA6AFB25E96EFC51EA22EF5097
:1035C000700817E14ACBE9FF4BCBEAFF0B014F51E3
:1035D000EF120B014C514C07000901E0FAD70B0127
:1035E0004F1D106E4ACBE9FF4BCBEAFF1050EF1690
:1035F0001DD0FDC0E9FFFEC0EAFFEF50310816E123
:103600000B014F1D106E4ACBE9FF4BCBEAFF105068
:10361000EF160B014C514C07000901E0FAD74ACBD9
:10362000E9FF4BCBEAFF0B014F51EF1283D1FBC0F7
:10363000E9FFFCC0EAFFEF506C0866E10001FF51B2
:1036400062E0010E0001EA6AFB25E96EFC51EA2204
:10365000EF506E0A21E00F0A11E0030A01E053D097
:103660000201080EC06FFDC0BEF2FEC0BFF23E0EEA
:103670000201BC6FBD6B5EEC31F045D00201080E5B
:10368000C06FFDC0BEF2FEC0BFF2350E0201BC6FBE
:10369000BD6B5EEC31F037D00B01010E4C6F0B01AE
:1036A0004D6B0F0E0B014D5D27E20B014C510AE0F3
:1036B0000B014D510001EA6AFD25E96EFE51EA2237
:1036C000EFCF4CFB0B014C510AE1200EA86E470EC8
:1036D0000B014D250001F06F0BEC38F009D04CCBFD
:1036E000A8FF470E0B014D250001F06F0BEC38F0E1
:1036F00004000B014D2BD5D7A86A0001560EF06FC0
:103700000BEC38F000D016D1FBC0E9FFFCC0EAFF9B
:10371000EF506D081AE10001FF5116E0FDC0E9FF0E
:10372000FEC0EAFFEF50720A01E00ED0D8EC20F0A4
:10373000FF0E986E966E956E936E000E866E846E7A
:10374000836E816EFF0000D0F5D0FBC0E9FFFCC0A6
:10375000EAFFEFCF10F0770E105C01E2EBD0010E24
:103760000001EA6AFB25E96EFC51EA22EF50660887
:103770001CE1FDC0E9FFFEC0EAFFEF50D00F0B01D6
:103780004C6F020E0001EA6AFB25E96EFC51EA2249
:10379000EF50720802E0000E01D0010E0001F76F39
:1037A0004CCBF6F038EC39F0C5D0010E0001EA6AD6
:1037B000FB25E96EFC51EA22EF50650821E1020188
:1037C0004C0EBA6F0B0EBB6FFDC0B8F2FEC0B9F263
:1037D00039EC31F0000913E0020E0001EA6AFB2522
:1037E000E96EFC51EA22EF50720802E0000E01D0AF
:1037F000010E0001F96F4CCBF8F07EEC39F09AD055
:10380000010E0001EA6AFB25E96EFC51EA22EFCFC6
:1038100010F0310E105C37E3010E0001EA6AFB255F
:10382000E96EFC51EA22EF5035082DE3FDC0E6FFBA
:10383000FEC0E6FF47EC44F0E552E552F3CF56FBFD
:10384000F4CF57FB020E0001EA6AFB25E96EFC513A
:10385000EA22EF50720802E0000E01D0010E0001D2
:10386000F46F56CBF2F057CBF3F0010E0001EA6A89
:10387000FB25E96EFC51EA22EF50D00F0001F16FF9
:10388000B4EC38F057D0010E0001EA6AFB25E96E6E
:10389000FC51EA22EF506D084DE10B01010E4D6F16
:1038A0000001650EEF6FFEEC37F0FE0B0B014C6F65
:1038B000FDC0E9FFFEC0EAFFEF50380808E13F0E07
:1038C000CB5C04E00B014D6B3F0ECB6E14D0FDC002
:1038D000E9FFFEC0EAFFEF5061080DE1CB50106E2A
:1038E000116AFF0E101801E1115003E00B014D6B3E
:1038F000CB680B014C810B014D510BE10001F76BC3
:103900000001640EEF6FFEEC37F00001F66F38EC4B
:1039100039F0020E0001EA6AFB25E96EFC51EA2249
:10392000EF50720807E14CCBA8FF0001650EF06F65
:103930000BEC38F048CBF3FF49CBF4FF00D012007A
:10394000EA6A030FE96E0B0EEA2212000251106EB2
:0C395000116A3F0E105C000E11581200AE
:04395C00966A868859
:1039600098880201806B816B826B836B846B856BA3
:103970000B01006B030E005D15E20051040DF3CF47
:1039800010F0F4CF11F0400E1026000E112200515D
:1039900046EC21F010C0EFFF00518EEC21F0EF80DB
:1039A000002BE8D7236A02017E69D8EC20F05EEC98
:1039B00021F002011F0E5BEC21F00201A16F020158
:1039C0001F0E58EC21F05EEC21F00201210E53ECA9
:1039D00021F05EEC21F00201080EA16F02010E0E33
:1039E0008BEC21F00A0E8BEC21F00B0E9CEC21F0FD
:1039F000040EA16F02010C0E9CEC21F0020EA16FCF
:103A000002010D0E58EC21F0AEEC21F058EC21F043
:103A100086EC21F0010E9CEC21F0600EA16F0201FA
:103A2000020E58EC21F086EC21F0030E9CEC21F004
:103A3000A1690201070E8BEC21F00F0E9CEC21F026
:103A4000610E53EC21F0D5C0A1F20201010E58EC39
:103A500021F0D6C0A1F20201020E58EC21F0D7C02D
:103A6000A1F20201030E58EC21F0D8C0A1F202012C
:103A7000040E58EC21F0D9C0A1F20201050E58EC59
:103A800021F0DAC0A1F20201060E58EC21F00B0180
:103A9000006B080E005D0BE20201A169080E0B012C
:103AA0000025020158EC21F00B01002BF2D786EC27
:103AB00021F0070E58EC21F04C0E206E0201220E70
:103AC00053EC21F074EC21F00D0E9CEC21F0E00E93
:103AD00053EC21F00201C00EA16F0201010E8BEC2C
:103AE00021F0040E8BEC21F0010E9CEC21F0200E55
:103AF00053EF21F002010D0EA4EC21F0020180270A
:103B00001150812302010E0EA4EC21F00201822744
:103B10001150832302010F0EA4EC21F0020184272F
:103B20001150852312000201865104E0CCDB01E034
:103B3000000C010C7E51235C04E1C5DB01E0000CAC
:103B4000010C0B01010E2B6F030E2B5D07E22B51B5
:103B5000B5EC21F001E0010C2B2BF6D7000C020193
:103B6000875104E0B0DB01E1000CFF0C0B01010EFA
:103B70002B6F030E2B5D0EE22B51B5EC21F008E00C
:103B80002B51CCDBEF902B51C9DBEF922B51120064
:103B90002B2BEFD7FF0CACDB86A8FED799DB86A8D2
:103BA000FED7ADDB86A8FED78D8C670E8D6E400EDE
:103BB000836E8D9C86A8FED78D8C700E8D6E88C20C
:103BC00083FF8D9C86A8FED78D8C212A000E222291
:103BD000120002018B518C1101E11200010E8B15B4
:103BE000106E116A8B5110240B01416F02018C5130
:103BF00011200B01426F956A670E8D6E400E836E29
:103C00008D9C86A8FED78D8C6A0E8D6E41CB83FF6E
:103C10008D9C86A8FED78D8C6B0E8D6E42CB83FF5C
:103C20008D9C86A8FED76BDB86A8FED78D8C020103
:103C30008B5121268C512222700E8D6E72DB86A84C
:103C4000FED78D8C8BC23FFB8CC240FB0B01010E5B
:103C50003F5F000E405B0B013FCB10F040CB11F0FB
:103C60003F07000E405B1050111030E0080E3F5D22
:103C7000000E405926E314DB86A8FED78D8C10DB9E
:103C800086A8FED78D8C0CDB86A8FED78D8C08DB32
:103C900086A8FED78D8C04DB86A8FED78D8C00DB32
:103CA00086A8FED78D8CFCDA86A8FED78D8CF8DA34
:103CB00086A8FED78D8C080E0B013F5F000E405B7F
:103CC000D5D7EEDA86A8FED78D8CC5D7120010DBCB
:103CD00086A8FED7FDDA86A8FED78D8CFF0E215C64
:103CE0001DE15F0E225C1AE10B01A669A769A6CB54
:103CF000A3F2A7CBA4F285DAF1DA86A8FED78D8CE1
:103D00000201100ED8DA0B01A56FA66B4C0EA76F3F
:103D1000A6CBA3F2E8CFA4F274DA10D0DFDA86A83B
:103D2000FED78D8C9568700E8D6E8D9A86A8FED705
:103D300083CFA5FB8D8A212A000E22220B01A551DB
:103D400012008FC2A5FB90C2A6FB02018F519011F9
:103D500003E1F36AF46A1200956A6A0E8D6EA5CBD0
:103D600083FF8D9C86A8FED78D8C6B0E8D6EA6CBA7
:103D700083FF8D9C86A8FED78D8CB0DA86A8FED7EF
:103D80008D8C0B01A5512126A6512222600E225CAA
:103D900002E3140E225E9568700E8D6E0B01A5CBAA
:103DA00010F0A6CB11F0A507000EA65B1050111065
:103DB0000FE08D9A86A8FED702018DC2E9FF8EC260
:103DC000EAFF8D2B000E8E2383CFEFFF8D8AE6D77F
:103DD0008FC2F3FF90C2F4FF120093C28CFB0B0161
:103DE0008D6B0201935103E1F36AF46A1200956A44
:103DF0006A0E8D6E93C283FF8D9C86A8FED768DA0B
:103E000086A8FED78D8C6ADA86A8FED78D8C956839
:103E1000700E8D6E0B018C512DE08C078D9A86A84B
:103E2000FED783CF8EFB8D8A02019151921109E05A
:103E300091C2E9FF92C2EAFF912B000E92238ECB32
:103E4000EFFF94510B018E5DE5E1200E8D6F956AB9
:103E5000600E8D6E200E836E8D9C86A8FED78D8C95
:103E60006A0E8D6E836A8D9C86A8FED731DA86A88D
:103E7000FED78D8C0B018C510201935D0B018C6F71
:103E8000E850106E116AE850212611502222600E6F
:103E9000225C02E3140E225E200E8D5D05E121C03E
:103EA000A3F222C0A4F2ADD9126A0B018C51000119
:103EB0001210F36E8DCBF4FF1200020195512EDA31
:103EC000EF901200030E0201965D05E2965126DA8C
:103ED000EF8096C223F0120020C0AAFB0B01010E56
:103EE000A96FE8CFA3F220C0A4F28BD9F0DE0B01BA
:103EF000A86FE8CFA1F20201030E58EF21F01FDAFC
:103F00000B01006F0201200ECED920500B01005D85
:103F100005E2600ED8802054002502D02050005DBC
:103F2000016FE850106E116A140ED8801056000E02
:103F3000115610C001FB10C003FB026B02CBF3FF54
:103F400010C0F4FF12000201E00E03DA0B01006F53
:103F50000201200EA8D90B010051040B01E0000C56
:103F6000010C99C2E9FF9AC2EAFFEF68E8D90B0198
:103F7000126F0201200EEDD90B01136FFAD9100B4D
:103F800034E0A1D90B01166F0201210E8CD9030177
:103F9000020EDC6F89EC4AF0A7D90A0EBCD90B0ED1
:103FA00087D90B01165108E0E4D90A0B02E0000E94
:103FB00001D0010E0B01166F0201020EA16F02016A
:103FC0000D0EBAD9220E6FD912CB20F085DF020177
:103FD000A1690201070E9FD90D0E6AD90B01165176
:103FE00003E00201260E5FD9000C0B011351125D94
:103FF00067E013CB15FB146B14CBA3F213CBA4F225
:1040000000D9120E02018F6F906B0201000E8D6FAE
:104010000B0E8E6F96DE0B010051010B4EE0400E31
:10402000025D000E035949E3EE0ED8800255050EDD
:10403000035543E3600E015D40E20151106E116AC9
:10404000D890115004E64C0E105C000E115835E368
:1040500010CBABF211CBACF21FEC30F0F3CF10FB76
:10406000F4CF11FB060EE66EE66A0A0EE66E0B0E44
:10407000E66E97C2E9FF98C2EAFF97C210F098C2B5
:1040800011F097C2E6FF98C2E6FF66EC47F0126EA9
:10409000060EE15E1250080E0B01115D0BE110518E
:1040A00003E0060E105D06E199C2E9FF9AC2EAFF3D
:1040B00010CBEFFF13CB20F0010C12CB20F00CDF64
:1040C000000C02010A0EA16F0201070EF1D8235065
:1040D000DDD8EFCF44FB0B01436B43CBA3F244CBC2
:1040E000A4F28FD8060E02018B6F8C6B9BC289F2F3
:1040F0009CC28AF26EDDD5C088F24DDDD6C088F252
:104100004ADDD7C088F247DDD8C088F244DDD9C087
:1041100088F241DDDAC088F23EDD02019D5103E103
:104120000B01456B03D00B01060E456F0201080E13
:10413000886F31DD45CB88F22EDD0E0E02019E2701
:10414000000E9F233C0E9E5D000E9F5903E23C0E25
:104150009E6F9F6B9EC243FB9FC244FB9EC2A1F217
:104160000201050EA5D844CBA1F20201060E58EFBC
:1041700021F0F4D8E1D8240E96D823C07EF2235043
:10418000CDD8EF802350CAD8EF820B012B6B030EE2
:104190002B5D0DE22B51E9D807E02B5102017E5D2A
:1041A00003E02BCB23F012000B012B2BF0D71200D6
:1041B0009568600E8D6E8D8C8D8A8D8E966A03014A
:1041C000010EDB6F7CEC4AF079D88D9E1200600EF8
:1041D0000201A0118D6EA1C283FF956A8D9C86A8F5
:1041E000FED78D8C12009568600E0201A2118D6EB3
:1041F0008D9A86A8FED783CFABFB8D8A0B01AB517E
:104200001200A3C221F0A4C222F0A3C2A1F20201B3
:10421000080E4ED8A4C2A1F20201090E58EF21F0F7
:104220000201090E48D80B01016F0201080E43D8A4
:10423000F36E01CBF4FF120020C093FB0B01120EB2
:10424000926F0201A5510B0192270201A6510B01A9
:10425000932392CBA3F293CBA4F201EF21F0A7C258
:1042600023F0235013D8EFCF2CFB0B010E0E2B6F36
:104270000201A8510B012B270201A9510B012C238C
:104280002BCBA3F22CCBA4F201EF21F0E96EEA6A6A
:10429000D890E936EA36780EE926020EEA221200B4
:1042A000020191EF21F0A16F0201A06BE7EF20F076
:1042B000A06FE7EF20F0A26FF3EF20F00301050EEF
:1042C000DC6F89EF4AF00201A26B8DDF040B120054
:1042D0008D8C6B0E8D6E836A8D9C1200600E8D6EC0
:1042E0000A0E836E8D9C12000201A16B0201120066
:1042F000956A6A0E8D6E010E836E8D9C12008D8CF8
:10430000600E8D6E120E836E8D9C120002014C0E9B
:10431000A16F02011200CCDF74EF21F0B7DFEE5283
:10432000120089C2E9FF8AC2EAFF892B000E8A23A4
:10433000EF50836E8D9C1200BBDF02011200020160
:10434000600EB1DFB9EF21F0B6DF106E116AE850F0
:104350001200A9DF0201030E5BEF21F0235096DF6C
:10436000EFCFA1F20201040E1200D8DFEF50010BD3
:0A43700012000201070E5BEF21F0BE
:06437A00080E0301D75DEF
:1043800001E11200FF0ED85D04E0D8C3B7F03CECA9
:1043900026F00301D869D76BDA6BD991D995120051
:1043A0000301D751070A01E1E5D0010A01E1A4D0D8
:1043B000030A01E192D0010A01E17ED0070A3AE046
:1043C000010A30E0030A08E0010A01E012000101DD
:1043D000EF6BF06BF16BF26B0101030EFE6F0B01E3
:1043E0000F691069116912691369146915691669F1
:1043F00017691869430E0001B56FB66B00010F0E07
:10440000B36F0B0EB46F440E0001B16FB26BEFECE3
:1044100025F00301D86FFF0ED85D01E11200B1DB7A
:10442000020ED76F9FDB140E105C000E115801E2D4
:10443000BCD044D001013C0EEB6FEC6BED6BEE6B2E
:10444000FE51FE07000922E1A1DB070ED76FD981DB
:10445000DA2BD9850001EF6BFEEC37F00001D16F4C
:104460000001010EEF6FFEEC37F00001D26F00018A
:10447000020EEF6FFEEC37F00001D36F0001030E68
:10448000EF6FFEEC37F00001D46F12000301D9A1E9
:1044900002D0050E2FD0D8C3B8F04FEC26F000099B
:1044A00001E183D00101010EFF6FBBDA0101FB6B5B
:1044B00068DB0301040E1ED077DB03E30301030E68
:1044C00019D0D8C3BEF06FEC27F000096EE06ED8AB
:1044D00002086BE10301050ED76FD8C3B8F04FECAB
:1044E00026F0000962E00101030EFF6F9ADA49DB52
:1044F0000301060ED76F1200D8C3BEF06FEC27F091
:10450000000932E053D80B01196F060E195D02E164
:10451000BDEF21F0050E195D2CE138DB32DB070E13
:10452000D76F0101FBA108D0EFC1D1F0F0C1D2F0EB
:10453000F1C1D3F0F2C1D4F0FBA508D0F7C1DBF094
:10454000F8C1DCF0F9C1DDF0FAC1DEF0FBA308D060
:10455000F3C1DFF0F4C1E0F0F5C1E1F0F6C1E2F043
:104560000301D981DA2B12001FDB1FE30301030EC5
:10457000D76F1200D9B51200F5DA640E105C000E88
:10458000115813E3EB07000EEC5BED5BEE5BEB51B8
:10459000EC11ED11EE1103E10301010ED76F640E72
:1045A0000101FC27000EFD23E7D712000B01036B6E
:1045B0000001000EBF6F0B0EC06F7EEC27F0020EE5
:1045C0000B01005D01E0FDD10B01016B0F0E0B0132
:1045D000015D0AE20001000EBF6F0B0EC06F7EECA2
:1045E00027F00B01012BF2D70301D9A311D00B0146
:1045F000016B040E0B01015D0AE20001000EBF6FAA
:104600000B0EC06F7EEC27F00B01012BF2D71ED0F2
:104610000001EF0EBF6F010EC06F7EEC27F00001AE
:10462000F00EBF6F010EC06F7EEC27F00001F10E9F
:10463000BF6F010EC06F7EEC27F00001F20EBF6F5E
:10464000010EC06F7EEC27F00101FB810B01016BB5
:10465000080E0B01015D0AE20001000EBF6F0B0E98
:10466000C06F7EEC27F00B01012BF2D7D5C009FB00
:10467000D6C00AFBD7C00BFBD8C00CFBD9C00DFBC2
:10468000DAC00EFB0B01016B060E0B01015D16E299
:104690000001000EBF6F0B0EC06F7EEC27F00B0108
:1046A0000151EA6A090FE96E0B0EEA22EF500B0185
:1046B000005D01E0B1D10B01012BE6D70B01016BCD
:1046C000CE0E0B01015D0AE20001000EBF6F0B0E62
:1046D000C06F7EEC27F00B01012BF2D70B01046BAE
:1046E0000001000EBF6F0B0EC06F7EEC27F00009BB
:1046F00004E10B01010E046F64D10B010051330A78
:1047000001E1E9D0CC0A01E1E2D0C90A01E1B5D06A
:10471000350A63E0020A21E0340A01E039D10001E0
:10472000000EBF6F0B0EC06F7EEC27F00B01000573
:1047300012E10001030EBF6F0B0EC06F7EEC27F07D
:1047400003010301D951020B05E0020E0B01035DC9
:1047500001E162D101D060D12FD10001000EBF6F05
:104760000B0EC06F7EEC27F0040E0B01005D33E1F1
:104770000301D9A311D00B01016B040E0B01015DE4
:104780000AE20001000EBF6F0B0EC06F7EEC27F037
:104790000B01012BF2D71ED00001F70EBF6F010EE7
:1047A000C06F7EEC27F00001F80EBF6F010EC06FE6
:1047B0007EEC27F00001F90EBF6F010EC06F7EEC9A
:1047C00027F00001FA0EBF6F010EC06F7EEC27F0DC
:1047D0000101FB8501D020D1EFD00001020EBF6F97
:1047E0000B0EC06F7EEC27F0040E0B01025D33E36D
:1047F0000301D9A311D00B01016B040E0B01015D64
:104800000AE20001000EBF6F0B0EC06F7EEC27F0B6
:104810000B01012BF2D71ED00001F30EBF6F010E6A
:10482000C06F7EEC27F00001F40EBF6F010EC06F69
:104830007EEC27F00001F50EBF6F010EC06F7EEC1D
:1048400027F00001F60EBF6F010EC06F7EEC27F05F
:104850000101FB8301D0E0D0040E0B01025F0B01CC
:1048600002510207000908E00001000EBF6F0B0EA5
:10487000C06F7EEC27F0F3D79FD00001000EBF6F12
:104880000B0EC06F7EEC27F0040E0B01005D1DE1E6
:104890000001080EBF6F0B0EC06F7EEC27F0000109
:1048A000070EBF6F0B0EC06F7EEC27F00001060EE7
:1048B000BF6F0B0EC06F7EEC27F00001050EBF6FBF
:1048C0000B0EC06F7EEC27F001D0A6D075D00B0187
:1048D000010E046F71D00001000EBF6F0B0EC06F90
:1048E0007EEC27F0040E0B01005D50E10301D9A31B
:1048F00011D00B01016B040E0B01015D0AE20001F6
:10490000000EBF6F0B0EC06F7EEC27F00B01012B6A
:10491000F2D73BD00001EE0EBF6F010EC06F7EECF0
:1049200027F00001ED0EBF6F010EC06F7EEC27F087
:104930000001EC0EBF6F010EC06F7EEC27F000018E
:10494000EB0EBF6F010EC06F7EEC27F0D880080E13
:104950000101EB55070EEC55000EED55000EEE551E
:1049600014E2EBC1EBF1ECC1ECF1EDC1EDF1EEC104
:10497000EEF1080E0101EB5F070E0101EC5B000E8A
:104980000101ED5B000E0101EE5B01D045D014D0BA
:104990000001020EBF6F0B0EC06F7EEC27F00B0103
:1049A00002510207000908E00001000EBF6F0B0E64
:1049B000C06F7EEC27F0F3D704000B01045101E136
:1049C0008FD6020E0B01035D0BE105CBE7F106CBA1
:1049D000E8F107CBE9F108CBEAF10301D98317D05D
:1049E000E70EE96E010EEA6EEE500B0105190CE1BF
:1049F000EE500B01061908E1EE500B01071904E116
:104A0000EE500B01081900E102E00B01036BCCEC46
:104A100027F00B01035104D0CCEC27F0000E00D09E
:104A200012000001010E99D8010E97D8060E95D8F4
:104A3000A3D8120E92D8230E90D8340E8ED8560ECC
:104A4000B9D8800EB7D898D897D8B96B5BEC26F058
:104A50000B01006B0C0E005D02E29FD8FBD7D5C0A6
:104A6000B9F05BEC26F0D6C0B9F05BEC26F0D7C00D
:104A7000B9F05BEC26F0D8C0B9F05BEC26F0D9C0F9
:104A8000B9F05BEC26F0DAC0B9F05BEC26F00B0174
:104A9000006BCA0E005D02E280D8FBD70001630EF6
:104AA0005CD8820E5AD8530E58D8630E56D8350E9D
:104AB00054D8010EB96F5BEC26F0FFC1B9F05BEC86
:104AC00026F00101FF0502E10301D9930101FF0571
:104AD00018E0EF51F011F111F21113E00001360E60
:104AE0006DD8EAC1B9F05BEC26F0E9C1B9F05BEC36
:104AF00026F0E8C1B9F05BEC26F0E7C1B9F05BEC59
:104B000026F00001370E29D8040E27D8010E25D82B
:104B1000030E23D8060E21D80C0EB96F5BEC26F0DD
:104B2000030E0101FF5D13E10001320E47D8EFC112
:104B3000B9F05BEC26F0F0C1B9F05BEC26F0F1C106
:104B4000B9F05BEC26F0F2C1B9F05BEC26F00001A5
:104B5000B9695BEC26F0D8EF26F0B96F5BEC26F074
:104B6000000112000101FC510301CC5D106ECD511A
:104B70000101FD55116E1200B96B5BEC26F00001CE
:104B80001200CCC3FCF1CDC3FDF11200D8C3B7F0C5
:104B90003CEC26F00301D86912000001B96B5BEC14
:104BA00026F00B01002B1200DDDF900E105C010ED1
:104BB00011581200D2DFE0DFBCEF25F0CEDF040E8B
:064BC000B96F5BEF26F067
:0A4BC6000B01006B040E005D06E217
:104BD00000CBB7F051D80B01002BF7D712000B0117
:104BE000600E226F000E236F216B040E215D43E2E5
:104BF00041DB0C0E31DB39DB126A136A10501110E5
:104C00001210131032E136DB0C0EB1C0EBFF0D0EAB
:104C1000B2C0EBFF0001B351B41111E00A0EE66E11
:104C2000E66AB3C0E6FFB4C0E6FF24DB22CB10F097
:104C300023CB11F022CBE6FF23CBE6FF2FDB1ADBE1
:104C40000A0EB5C0EBFF0B0EB6C0EBFF13DB0E0E6A
:104C5000EB6A0F0EEB6A0EDB100EEB6A110EEB6ABD
:104C600021CBB0F00B0121511200140E2227000EAF
:104C70002323212BBAD7FF0C0001B751E3DA0C0E26
:104C8000EBDAEE6AED6AB751DDDA060EE5DAEE6AC6
:104C9000EE6AEE6AEE6AB75129DBEF901200040E5D
:104CA0000001B85D07E2B8C0B0F00201010E866FE6
:104CB00093EF1DF0000C0001B051140DF3CF46FB33
:104CC000F4CF47FB600E0B014627000E472316DB8F
:104CD000EE50ED100FE1E9DAD2DA14DBD0DA120E81
:104CE000EB50FF0801E1000C1C0E0201A86FA96B3C
:104CF000C6DAE2DAB9C088F2CBEC1DF0FFDAEE2AB0
:104D0000EF22FCDA05DB01E353D8010C0001B051BE
:104D1000140DF3CF00FBF4CF01FB600E0B01002755
:104D2000000E0123E7DAEE50ED1011E1BEDA98DA59
:104D3000E9DA96DA120EEB50FF0803E1F36AF46A3F
:104D400012001C0E0201A86FA96B8ADAB5DAD2DA5A
:104D50000001BC51EE24106EBD51EE20116ED60E36
:104D6000D8801054030E11540AE2C4DAEECFBCF01E
:104D7000EFCFBDF0D60ED880BC57030EBD57BCC0D8
:104D80008BF2BDC08CF2BAC089F2BBC08AF2E9ECEA
:104D90001DF0B0DA0001BC51EE26BD51ED22AADAB9
:104DA000B7DA01E305D8BCC0F3FFBDC0F4FF1200C1
:104DB0000201010E866F93EC1DF0000902E1040070
:104DC000F7D70001B051140DF3CF29FBF4CF2AFB24
:104DD000600E0B012927000E0B012A2329CBE9FFC6
:104DE0002ACBEAFF0C0EE926000EEA22EECFABF248
:104DF000EDCFACF21FEC30F0F3CF21FBF4CF22FB70
:104E000029CBE9FF2ACBEAFF0A0EE926000EEA22A7
:104E1000EECFABF2EDCFACF21FEC30F0F3CF23FBD3
:104E2000F4CF24FB29CBE9FF2ACBEAFF0E0EE926BB
:104E3000000EEA22EECF25FBEFCF26FB080E0B017A
:104E40002527000E0B0126230B01276B286B140E60
:104E50000201A86FA96B29CBE9FF2ACBEAFF120E4A
:104E6000EB500201A76F2FEC21F025CB6EF326CB80
:104E70006FF30301110E6D6F29CBE9FF2ACBEAFF17
:104E8000E9CF6BF3EACF6CF3DAEC3FF025CBABF272
:104E900026CBACF21FEC30F0F3CF25FBF4CF26FB92
:104EA000080E02018B6F8C6B0201210E896F0B0EB5
:104EB0008A6FE9EC1DF0B9EC20F029CBE9FF2ACB91
:104EC000EAFF120EE926000EEA22EF6829CBE9FF7D
:104ED0002ACBEAFF0E0EEB6A0F0EEB6A1200040EED
:104EE0000001BE5D0AE2BEC0B0F0FBD9D880EE542E
:104EF000000EED5401E3000C010C000C13DA01E18B
:104F0000000CB051F3D9EF50010B01E00FDA67EC60
:104F10001EF0BFC0E9FFC0C0EAFFEF6E0DDAEE067B
:104F2000EF5ADFD9EE50ED1002E16CEC1FF0010CEE
:104F3000F9D903E1F36AF46A1200B051D7D9EF50FE
:104F4000010B01E0F3D9F8D990D9C351105CC451D9
:104F5000115805E2C6D9EECFC3F0EDCFC4F0C3C0FF
:104F60008FF2C4C090F2C1C08DF2C2C08EF2A1EC2B
:104F70001EF0F3CF00FBF4CF01FBDED90B01005193
:104F8000EE5E0151ED5ACED902E16CEC1FF0C3C0C8
:104F9000F3FFC4C0F4FF1200C5D902E06CEC1FF0AF
:104FA000CBD9EE6AED6A1200080E02018F6F906B8A
:104FB0000201460E8D6F0B0E8E6FA1EC1EF046CBDC
:104FC0005DFB47CB46FB5DCB47FB48CB5DFB49CB4D
:104FD00048FB5DCB49FB080E106E0B014B51D8808E
:104FE000105403E24A055D6F02D04ACB5DFB080E08
:104FF0004B5D4A6F5DCB4BFB4C514D116AE04CCB86
:105000005DFB4DCB4CFB5DCB4DFBC5C0E9FFC6C086
:10501000EAFF060E21D9EECF4FFBEECF50FBEECFCD
:1050200051FBEFCF52FB4ED9EFCF53FB010E14D9FA
:10503000EFCF54FB47D9020E0FD9EFCF55FB42D922
:10504000030E0AD9EFCF56FB576B110E586FC9C02C
:1050500059FBCAC05AFBC9C0ABF2CAC0ACF21FECC4
:1050600030F0F3CF59FBF4CF5AFB0C0E0201B36FB3
:10507000B46B02014F0EB16F0B0EB26F53EC30F0F8
:10508000F3CF5BFBF4CF5CFB0B015B1F5C1F060ED9
:1050900000D95BCB88F2CBEC1DF0070EFAD85CCBC5
:1050A00088F2CBEC1DF00301706B716B49EC40F0A2
:1050B000C9C0B5F2CAC0B6F2BFEC30F0F3CF5BFBAB
:1050C000F4CF5CFB0B014C51F31816E14D515C1908
:1050D00013E1C7C0CFF0C8C0D0F0C5C0CDF0C6C086
:1050E000CEF00001460ECB6F0B0ECC6F1CD80B011F
:1050F0004E6FFF0E4E5D03E16CEC1FF0010C4E5144
:10510000A1D8100EA9D84ACBEEFF4BCBEDFF4E51E4
:10511000EDD8EF80010C0001B05194D8E9CFF3FF36
:10512000EACFF4FF12000B010169600E026F000E5E
:10513000036F006B040E005D5BE2A6D80C0EEED888
:10514000020E8AD8C9D80001125010184AE1135033
:10515000111847E199D80A0EE1D8BED8125010189C
:105160003EE1135011183BE18FD8100E75D8EECFE9
:1051700014F0EFCF15F0166A176A145015101610B8
:1051800017102DE1CDC0E9FFCEC0EAFF060E64D8AE
:10519000EECF10F0EECF11F09FD876D8060E5CD887
:1051A000EE50101808E1EE50111805E1EE501218FB
:1051B00002E1EE50131810E0CFC0E9FFD0C0EAFFC3
:1051C000E868EE180CE1E868EE1809E1E868EE1806
:1051D00006E1E868EE1803E10B010051120000CB74
:1051E00001FB0B01140E0227000E0323002BA2D794
:1051F000FF0E015D24E00151140DF3CF02FBF4CF4B
:1052000003FB600E0227000E03230A0EE66EE66A19
:10521000CDC0E6FFCEC0E6FF37D802CB10F003CBFF
:1052200011F002CBE6FF03CBE6FF38D850D81DD8EB
:105230002BD80A0E10C0EBFF0B0E11C0EBFF0B01B9
:1052400001511200140DF3CFE9FFF4CFEAFF600E15
:10525000E926000EEA221200E926000EEA221200D8
:1052600000CBE9FF01CBEAFF1200EECF10F0EFCF49
:1052700011F0120022CBE9FF23CBEAFF120046CB4C
:10528000E9FF47CBEAFF120002CBE9FF03CBEAFFBD
:1052900012000301706F716B49EF40F066EC47F04C
:1052A000126E060EE15E125012000201010E876FAF
:1052B000AFEC1DF0E66E1200120EEB500201A76F6C
:1052C0002FEF21F0C7C0E9FFC8C0EAFF1200CBC032
:1052D000E9FFCCC0EAFF1200EECF12F0EFCF13F0DF
:1052E0001200B051AFDF100E2CEF29F0ABDF130E20
:1052F0002CEF29F0B5DF0E0E2CEF29F0C0DF0E0EDB
:105300002CEF29F0120EA8DFE552E750EF6E1200E5
:10531000ACDFD60E105C030E115812009DDFA5DF26
:1053200067EF29F009D8EE50ED101200B051DEDF22
:0E533000EF90080E49EF29F0000171EF29F00F
:02533E0012005B
:105340004CDB040B05E049DB080B01E0020C010C0F
:10535000000C0B01406B416B446BE4C2E2F2E5C20E
:10536000E3F2EEDF0B01456F400E426F0F01420E7C
:10537000476F0B0E486F0F01000E456F0B0E466F07
:10538000E4C2E9FFE5C2EAFFEF500F01446F04EC0D
:1053900013F00B01436F442B476B6C0E005D08E16B
:1053A0000151750A02E0050A19E1010E476F16D096
:1053B0006D0E005D13E1455105E017DB6F0A02E158
:1053C000010E476F12DB6C0A09E1010E476FE4C260
:1053D000E9FFE5C2EAFF090E1CDBEF88475116E141
:1053E00045CBFFF042510001FD6FFE6B000EFD2723
:1053F0000B0EFE230001000EFB6F0B0EFC6FD3ECB7
:1054000017F0F3500B014013F45041134351ACE13A
:105410004051020B01E012004051040B02E02FEF5B
:1054200038F04051080B02E07EEF38F04051100B8D
:1054300002E0AAEF38F04151010B02E0ACEC39F088
:105440001200B0DA020EE5DAEFCF01FBABDA030EA1
:10545000E0DAEFCF02FBA6DAEECF07FBEDCF08FBD9
:10546000D3DAEF6AE8C2E2F2E9C2E3F269DF0B01E4
:10547000096F610E025D6CE30251680869E3006B1D
:10548000610E025D066F070E0115106E010E1052BF
:1054900004E0E846FE0B1006FCE10B01056F065127
:1054A000036F046B920E03270F0E042389DA09E1C0
:1054B0000651036F046B890E03270F0E042300812E
:1054C00007D00651036F046B800E03270F0E0423D1
:1054D000F00E0115066FE85004E172DA01E173D0B5
:1054E0006DD0100E065D0CE16BDA05E10201590E7C
:1054F000EF6F950E94D10201560EEF6F950E8FD17E
:10550000200E065D03E1010E001506E0300E065D7B
:1055100008E1010E001505E0080E011501E16AD150
:105520007AD1400E065D0CE101A703D000B19BD1FA
:1055300002D000A198D102013C0EEF6F950E6FD101
:10554000500E065D01E08FD1010E001537E03BD013
:105550006B0E025D0AE1095105E001CBEFF0FEECB4
:1055600037F060D00201FD6B5FD06C0E025D41E14F
:10557000010505E102011C0EEF6F960E50D1020EDF
:10558000015D05E10201CC0EEF6F950E48D1040ECE
:10559000015D05E102011C0EEF6F790E40D1015152
:1055A00008E1095101E04FD10201160EEF6F790EAB
:1055B00036D1030E015D04E1095105E0310E3ED103
:1055C000060E015D02E1300E39D1050E015D02E1EA
:1055D000470E3ED1100E015D01E245D10151210877
:1055E00001E241D1100E015DEA6AD10FE96E000EB1
:1055F00017D06E0E025D01E075D0006B0F0E011525
:10560000106EC11C0F0B105C01E20083F00E01153F
:10561000066FE85001E1CAD0100E065D07E1EDD932
:10562000EA22EF500201FD6FFE6BD0D0200E065D26
:105630003BE1E3D9EA22EFCF06FB0751081120E155
:10564000330EC5D90750300F0201DC6F2E0EDD6F0F
:10565000330EBDD903C006FB0B0103500A0D8ED9D2
:105660000201DE6F0A0EB3D907C006FB0B0107501B
:10567000640D84D90201DF6FE06B0B01076B086BCF
:10568000075197D9C1D9EF6E075193D901E1EBD0FA
:1056900007CB10F008CB11F0072B000E082307CB27
:1056A000F3FF08CBF4FF1200300E065D04E1020E9A
:1056B000001501E09FD0500E065D04E1020E0015BA
:1056C00001E198D0400E065D04E1020E001501E0F4
:1056D000A2D0600E065D01E0C6D0020E001501E00A
:1056E000C2D099D0770E025D01E0A2D0006B0F0E00
:1056F00001150B6F0A6BE80403E1BDCF0AFB11D063
:10570000020E0B5D03E1BACF0AFB0BD0030E0B5D5B
:1057100003E1B7CF0AFB05D0040E0B5D02E173CFA6
:105720000AFB0F0E0A1501E00087F00E0115066F47
:10573000F00E065D39E10B5104E168EC39F0300FF1
:105740007DD0040E0B5D11E1CB50106E116AFF0E7F
:10575000101801E1115002E0000E01D0010E010805
:1057600002E1610E6BD0380E69D0080E0B5D01E0CE
:105770007AD0066B0F0EBD1401E006810F0EBA142D
:1057800001E006830F0EB71401E006850F0E7314B7
:1057900001E0068706CBF9F2EAC2F7F2EBC2F8F2B3
:1057A00007CBF6F276EF2CF0065105E102012C0E44
:1057B000EF6F950E34D0100E065D10E10BCBF5F0B7
:1057C00003EC39F0F3CFFDF2F4CFFEF2EAC2FBF2C4
:1057D000EBC2FCF207CBFAF295EF2CF0300E065D2F
:1057E00003E1080E001506E1500E065D08E1080E03
:1057F000001505E102014D0EEF6F950E10D0400E21
:10580000065D03E1080E001506E1600E065D2BE162
:10581000080E001528E10201520EEF6F950EF06F91
:10582000EAC2EDF2EBC2EEF207CBECF236EF2CF06F
:10583000730E025D18E1095104E1300EE5D8EF6EF8
:1058400012D0015102E1350E03D001050CE13E0EEC
:105850000201F46FF56BEAC2F2F2EBC2F3F207CB8E
:10586000F1F255EF2CF0F368F46812000201EC51EC
:10587000F76AEF25F66EF051F7220800F550EDC2F9
:10588000E9FFEEC2EAFFEF6EEDC2E9FFEEC2EAFF0A
:10589000EF5003E1F368F4681200EC2BEC51116A4D
:1058A000ECC2F3FF11C0F4FF12000201F151F42524
:1058B0000B010C6F000E0201F521AA6E0CCBA9FFA3
:1058C0003F0EA616A680A850F2C2E9FFF3C2EAFF77
:1058D000EF6EA85003E1F368F4681200F12BF15168
:1058E000116AF1C2F3FF11C0F4FF1200020E0201AF
:1058F000F65D03E3F368F4681200F65103E1F93949
:105900000F0BF96F0F0EF915090802E2370E01D0DF
:10591000300EF925F7C2E9FFF8C2EAFFEF6EF6296B
:10592000116AF36E11C0F4FF12000201FA5111E185
:10593000DC0EE66E020EE66EFDC2E6FFFEC2E6FF7C
:10594000BCEC44F0E552E552E552E5520201E16B50
:10595000FA6BFA512ED8FBC2E9FFFCC2EAFFEF6EE8
:10596000FA5127D803E1F368F4681200FA2BFA51D0
:10597000116AFAC2F3FF11C0F4FF1200F3CF10F066
:10598000F4CF11F0330E0B6E0C6AF3CF06F0F4CFA8
:1059900007F0AFEC4AF006C010F007C011F0300E6F
:1059A00006241200E8C2E9FFE9C2EAFF040E09EF8B
:1059B0002DF0EA6ADC0FE96E020EEA22EF501200C7
:1059C00003CBE9FF04CBEAFFEF5005151200106E80
:1059D0000C6E06CB07F0F4EF4AF0E2C2E9FFE3C237
:1059E000EAFF090E16D8EF5012004251EA6A000F82
:1059F000E96E0B0EEA22EF5012000F0E0115EA6A53
:105A0000E30FE96E000E1200EAC2E9FFEBC2EAFF03
:0A5A10001200E926000EEA2212003F
:065A1A000F01525101E1F1
:105A200012000D01890EF96F8E0EFA6FE2EC48F04C
:105A30000D01AC0EF96F8C0EFA6FE2EC48F052CF0C
:105A4000A9FB0B01A951000817E2A951070B05E1B9
:105A50000D012E0EF56F82EC48F00D01F2510D0193
:105A6000F35D02E0E1D908D00301320EDC6F89EC6E
:105A70004AF00B01A907E5D70D01D40EF96F8C0E82
:105A8000FA6FE2EC48F00F01D10E536F000E546F25
:105A90004AEF2DF0BDDA89DA010EE926000EEA227E
:105AA00084DA020EE926000EEA227FDA030EE926E6
:105AB000000EEA22F8EF2FF00B01016B0D01F251FD
:105AC0000D01F35D02E10400F9D772EC48F00B011F
:105AD000006F0D0E0B01005D04E00A0E0B01005D6E
:105AE00001E118D00B01012B0F0155CFE9FF56CF73
:105AF000EAFF552B000E562300CBEFFF55CFE9FFF1
:105B000056CFEAFFEF6A0F0157515707000901E12D
:105B100001D0D4D70B01015100D0120058CF01FBA6
:105B200059CF02FB0B01036B58CFE9FF59CFEAFFB6
:105B3000EFCF00FBEF5021E02E0E0B01005D11E1D5
:105B40000F0158CFE9FF59CFEAFF582B000E592318
:105B5000EF6A33DA032B42DA58CF01FB59CF02FB4D
:105B600007D0300E005D03E30051390801E2000C5C
:105B70000F01582B000E5923D7D71FDA2FDA030E47
:105B80000B01035D01E0000C010C0D01F2510D0150
:105B9000F35D02E10400F9D772EC48F00B01006FED
:105BA000310E0B01005D08E3390E0B01005D04E2CC
:105BB0000B01005103D002D0390E00D012000D01AC
:105BC0000D0EF56F82EC48F00D010A0EF56F82ECB8
:105BD00048F0300E0F015C5DFF0FE96EEA6AD89065
:105BE000E936EA36850EE926030EEA22EECFF9FD04
:105BF000EDCFFAFDE2EC48F00F015C51380A01E10B
:105C000011D10F0A01E10CD1010A01E1FCD0030A14
:105C100001E1ECD0010A76E0070A6BE0010A61E0DD
:105C2000030A01E000D10001330EEF6FFEEC37F004
:105C30000B01A16F0001340EEF6FFEEC37F00B018A
:105C4000A26F870EE66E0B0EE66EA1CBE6FFA2CB2F
:105C5000E6FFBCEC44F0E552E552E552E5520D0199
:105C6000870EF76F0B0EF86FD0EC48F00D01290E80
:105C7000F56F82EC48F00D013A0EF56F82EC48F0BA
:105C80000D01200EF56F82EC48F00F01140E576FD6
:105C90000F01870E556F0B0E566F0EDF00091FE0C8
:105CA000870EE66E0B0EE66E47EC44F0E552E552C9
:105CB000F3CFA1FBF4CFA2FBA1CBA8FF0001330ED1
:105CC000F06F0BEC38F0A2CBA8FF0001340EF06FA0
:105CD0000BEC38F0A2CBD9F0A1CBDAF001D044D054
:105CE000A2D00B01D10E9F6F000EA06F0B01A36B12
:105CF00011D00B01DF0E9F6F000EA06F0B010E0E77
:105D0000A36F08D00B01DB0E9F6F000EA06F0B017D
:105D10000A0EA36F9FCB53FFA0CB54FFBBDE0D0138
:105D2000290EF56F82EC48F00D013A0EF56F82EC0A
:105D300048F00D01200EF56F82EC48F00F01140EB3
:105D4000576F0F01870E556F0B0E566FB5DE0F01A3
:105D50009B0E5A6F0B0E5B6F0F01870E586F0B0E69
:105D6000596FDCDE000911E10D013F0EF96F8E0E57
:105D7000FA6FE2EC48F00D01F2510D01F35D02E122
:105D80000400F9D772EC48F030D09FCBE9FFA0CBEC
:105D9000EAFF9BCBEEFF9CCBEEFF9DCBEEFF9ECBB5
:105DA000EEFF9BCBA8FF0B01A351A32B0001F06FCB
:105DB0000BEC38F09CCBA8FF0B01A351A32B0001E7
:105DC000F06F0BEC38F09DCBA8FF0B01A351A32B78
:105DD0000001F06F0BEC38F09ECBA8FF0B01A35134
:105DE000A32B0001F06F0BEC38F01DD00001160E54
:105DF000EF6FFEEC37F00109A86E0001160EF06F90
:105E00000BEC38F010D00001160EEF6FFEEC37F0FF
:105E1000FE0BA86E0001160EF06F0BEC38F003D0ED
:105E200018D801D000D012000D01090EF96F8D0EA7
:105E3000FA6FE2EC48F0A9DE0B01AA6F390EAA5DF9
:105E400003E0AACB5CFFBBDE380E0B01AA5DECE1E0
:105E500012000B01006B0B01026B51EC37F0CCC34D
:105E600085FBCDC386FB0B0185510301CC5D106E14
:105E7000CD510B018655116E320E105C000E11587B
:105E800009E3CCC385FBCDC386FB0D01150EF56F71
:105E900082EC48F004000D01F2510D01F35DE3E0E6
:105EA0000B01025101E07ED004000D01F2510D0101
:105EB000F35D05E072EC48F00B01016F01D0F0D703
:105EC0000B010051030A2EE0010A28E0030A1DE03D
:105ED00000D00B01010504E10B01010E006F14D08D
:105EE000040E0B01015D0BE193EC37F00D01060E82
:105EF000F56F82EC48F00B01010E026F05D00D0129
:105F0000150EF56F82EC48F04CD00B01060E046FB5
:105F10000B01036B0B01020E006F43D00B01030E4C
:105F2000006F3FD00B010351032BEA6A050FE96EA6
:105F30000B0EEA2201CBEFFF0B010351106E116A29
:105F4000113404E210508008000E115429E20B01B4
:105F5000060E046F0B01016B0B010151106E116AEB
:105F6000D890115004E6800E105C000E11580EE21D
:105F70000B010151EA6A050FE96E0B0EEA22EFCF21
:105F800045F269EC37F00B01012BE6D70201376BC4
:105F900090EC36F004CBF5FD82EC48F00B01006B81
:105FA00000D07ED7010E00D0120022D80D012E0E97
:105FB000F56F82EC48F008EF30F001CBE6FF02CB42
:105FC000E6FF47EC44F0E552E552F350E66E5ACF57
:105FD00010F05BCF11F00B01035112000F011024E0
:105FE000E96E000E1120EA6EE552E750EF6E1200E6
:105FF000EF50E66EE66ABCEC44F0E552E552E5523D
:10600000E5520D01000EF76F0B0EF86FD0EF48F060
:10601000000EE66E0B0EE66E53CFE9FF54CFEAFF9B
:0260200012006C
:0E6022000201AA390F0BAA6FE850090804E228
:10603000410EAA25F60F1200300EAA251200ACC29E
:10604000F3FFABC2F4FF1200ADC201FBAEC202FB14
:10605000AFC203FBB0C204FB0B01010E056F0B0EB8
:10606000066F05CBE9FFEA6E030EA1DAEF50E66E8C
:10607000030E97DA00CBEFFF73DA020E98DA010E07
:1060800087DAEF50E66E6CDA020E8BDA010E80DAF8
:1060900000CBEFFF01CB04F002CB05F003CB06F001
:1060A00004CB07F012000B01A96BAA6BAB6BAC6BB6
:1060B000B1C2A7FBB2C2A8FBB3C2A5FBB4C2A6FB88
:1060C000D890A633A533A5CB10F0A6CB11F0A50729
:1060D000000EA65B1050111018E0A7CBE9FFA8CB6B
:1060E000EAFF020EA727000EA823EECF10F0EFCF95
:1060F00011F0000110500B01A927000111500B01F4
:10610000AA23000EAB23AC23DED70201B351010B4F
:106110000EE0A7CBE9FFA8CBEAFFEFCF10F000011C
:1061200010500B01A927000EAA23AB23AC230B01AF
:10613000AB51AC1119E0A9CB10F0AACB11F0126A47
:10614000136AABCB14F0ACCB15F0166A176A10507B
:106150001424A96F11501520AA6F12501620AB6F8E
:1061600013501720AC6FE3D7A9CB10F0AACB11F0D6
:10617000101E111E10C0F3FF11C0F4FF12000B011E
:10618000010E006F016B026B0201B551B6114EE0BA
:10619000400EB55D000EB65904E3400E106E116A54
:1061A00004D0B5C210F0B6C211F010C005FB0B014F
:1061B000105002018F6F906B0201060E8D6F0B0E57
:1061C0008E6FA1EC1EF00B010551106E116A10507C
:1061D0000201B55F1150B65B0B01046B0551045D04
:1061E000D3E20451EA6A060FE96E0B0EEA22EFCF02
:1061F00003FB00510AE103510125016F0351015DC9
:106200000DE2022B0BE1012B09D003510225026F95
:106210000351025D03E2012B01E1022B005102E078
:10622000000E01D0010E006F042BD8D70B01021D08
:10623000026F011DF36E02CBF4FF12000201B75191
:10624000390805E3300EB75D02E3300E0FD0B751C9
:10625000460805E3410EB75D02E3370E07D0B7519C
:10626000660806E3610EB75D03E3570EB75D1200E3
:10627000FF0C010E0201EA6AB825E96EB951EA2263
:10628000EFCFB7F2DBDF0B01586FB8C2E9FFB9C23D
:10629000EAFFEFCFB7F2D2DF0B01596FFF0E585D67
:1062A00003E0FF0E595D01E1000C5939F00B581164
:1062B000BAC2E9FFBBC2EAFFEF6E010C0B01586BDB
:1062C000A6A202D00400FCD72F0EA616A6840201B7
:1062D000BEC2E9FFBFC2EAFFBE2B000EBF23EF50D4
:1062E000A86E0B01582B0201C0510B01D8805855E4
:1062F00001E2A86ABDC210F0116A1050AA6E020134
:10630000BCC210F0BDC211F0BC2B000EBD2310505A
:10631000A96E550EA76EAA0EA76EA6820000A6A2B1
:1063200002D00400FCD7A850D2E1A6940B01580576
:1063300000D012000B01CD6BA6A202D00400FCD746
:106340003F0EA6160B01CD2B0201C5510B01D880C3
:10635000CD5506E2C1C2E9FFC2C2EAFFEF6A18D01A
:10636000C3C2A9FFC4C210F0116A1050AA6E020184
:10637000C32B000EC423A680A850C1C2E9FFC2C22D
:10638000EAFFEF6E0201C12B000EC223A850DAE132
:106390000B01CD0500D01200C9C210F01050AA6E3A
:1063A000C8C2A9FF3F0EA6160201C6C2E9FFC7C2B6
:1063B000EAFFC62B000EC723EFCF48FBA680A850EC
:1063C0000B01485D01E0010C485101E1000CA92AD4
:1063D000EBE1AA2AE9D70201CAC2E9FFCBC2EAFF70
:1063E000CA2B000ECB23EFCFCDFBEF501FE0610E89
:1063F0000B01CD5D05E3CD517A0802E3200ECD5FA0
:106400000201CCC2F6FFCDC2F7FFCC2B000ECD238C
:106410000800F5500B01CD5D01E0000CCCC2F6FF89
:10642000CDC2F7FF0800F550D6E1010C000CCEC23A
:106430000CFBCFC20DFB0B010A6B0B6B0201D051A1
:106440000B010A5D0201D1510B010B590BE20CCB80
:10645000E9FF0DCBEAFF0C2B000E0D23EF6A0A2B90
:106460000B23ECD712001200030E0201DB5D37E3B1
:106470007CD8F6BEF7686AD8010E6CD8EF380F0BDF
:10648000106E7ED81010F66EF76AF6BEF7685ED80A
:10649000060E116E020E5ED8EF5011C0E7FFE752F4
:1064A00004E0E8427F0BE706FCE1106E010E0201FA
:1064B00083D81010F66EF76AF6BEF76847D8020E5A
:1064C00049D8EF503F0BF66EF76AF6BEF7683ED834
:1064D000030ED927000EDA23030EDB5FC5D7DB518D
:1064E00000082EE242D8F6BEF76830D849D80B0132
:1064F000CD6F0201DB51010806E2010E2BD8EF3807
:106500000F0B0B01CD130B01CD51F76A800FF66E07
:10651000940EF7220800F550E66E02013DD8020EF7
:10652000DB5D02E23D0E07D0010E46D8F66EF76A3B
:10653000F6BEF76847D8E66E2FD84BD83D0EEF6E03
:10654000D7C2E9FFD8C2EAFFEF6A12003BD8E66E75
:10655000CCEF32F0EA6AD925E96EDA51EA2212006C
:1065600005CBE9FF06CBEAFF1200D9C2E9FFDAC288
:10657000EAFFEF50E840E8403F0BF66EF76A120082
:10658000D9C2E9FFDAC2EAFFEF38F00B300B120094
:10659000E926000EEA2212001CD8E552E750EF6E01
:1065A0001200F6DFE552E750EF6EB0EF32F0F0DFA9
:1065B000EFCF00FBB0EF32F0CDDFEF50040DF35022
:1065C0003C0B1200800EF626940EF7220800F550C0
:1065D0001200D7C2E9FFD8C2EAFFD72B000ED8239A
:0265E0001200A7
:0E65E200150E0101536F546B89EC04F001019A
:1065F000A06FA46BD26B9F6B140EA26FA36B1200E3
:10660000A0C159F143EC05F0000908E10101D26B8A
:10661000080EA66FA46B9F6BA56B010CA0C172F155
:10662000E1EC07F0000935E052DA0101700E706FFD
:106630000B0E716FA0C16FF1A2EC07F000090FE023
:106640000101D251D22BEA6AB10FE96E010EEA22A2
:1066500070CBEFFF1F0ED25DE8E1D26BE6D7A0C191
:1066600064F1CFEC06F00A0E0B01705D27E1010129
:10667000D251EA6AB10FE96E010EEA22EF6AD26BDB
:10668000D3D9D3C1E5F1D4C1E6F195D90101A66F03
:1066900015D00101A45112E0E2510301CC5D106E4E
:1066A000CD510101E355116E500E105C460E11588C
:1066B00005E30DDA020EA66F010EA46F0101A451CD
:1066C000010A3AE0050A04E0040A54E1A76BFFD985
:1066D000A0C15CF1DFEC05F0000901E1010CA7C1EC
:1066E000E9FFEA6AE9BEEA68D890E936EA36340E8C
:1066F000E926030EEA22EECF71FBEDCF72FB0B0110
:1067000071CBF6FF72CBF7FF712B000E72230800DE
:10671000F5CF70FBF55007E070CB5EF1A0C15DF1E5
:1067200002EC06F0ECD7A0C15BF18FEC05F00101A3
:106730000C0EA76F010EA46F080EA65D1BE0A6C18C
:10674000E4F119D800090FE00C0E0101A75D03E088
:10675000040EA46F04D0020EA65D01E1A46B080E26
:10676000A66FA56B010C0C0E0101A75D03E0040EE2
:10677000A46FAED7010C0101E451060A54E0030AEC
:1067800050E0060A4CE0070A34E0060A30E0030A4B
:1067900018E0010A52E19F819F93010EA76F090E35
:1067A000E66EE66AD5C1E6FFD6C1E6FFA80EE66E44
:1067B000010EE66EEEEC47F0106E060EE15E105034
:1067C000010C9FA112D0D5C1ADF3D6C1AEF3030128
:1067D000A80EAB6F010EAC6F0CEC3FF0000904E0AB
:1067E00001019F83020E2AD00101060E27D020EF5F
:1067F00034F0DDC1E6FFDEC1E6FF47EC44F0E552D0
:10680000E552F3CFA3F1DFC1E6FFE0C1E6FF47ECBD
:1068100044F0E552E552F3CFA2F1010102D056EF68
:1068200034F00B0E0BD00B0EA76FFE0EA15D07E030
:10683000A1C15AF14CEC05F0010C050EA76F010C3B
:106840000101A551030A21E0020A14E0010A2DE129
:10685000020EA55D02E193EC37F0FE0E0101A15D91
:106860000FE093EC37F0A1C15AF14CEC05F00101B7
:10687000010E09D0A1C159F143EC05F0000915E161
:106880000101030EA76FA56F000CA0C15CF1DFEC46
:1068900005F000090AE0A0C159F143EC05F0000938
:1068A00004E0A0C15AF14CEC05F0000C0101A55127
:1068B000020A46E0030A35E0010A01E079D001014D
:1068C0009FB306D00101060EA76F010E73D028D02A
:1068D0000101070EA76FA2C157F1A3C158F1010131
:1068E000A051240DF3CFE9FFF4CFEAFF000EE92613
:1068F0000C0EEA22EE52E9CF55F1EACF56F1CEEC7A
:1069000004F00101A16FFE0E0101A15D04E001018F
:10691000010EA56F05D001010A0EA76F010E4AD026
:1069200047D0A1C159F143EC05F0000908E002018C
:1069300031A105D051EC37F00101020EA56F38D01E
:10694000A1C172F1E1EC07F000091EE0CCC3E2F155
:10695000CDC3E3F10101730E706F0B0E716FA1C116
:106960006FF1A2EC07F0000906E073CB45F269EC89
:1069700037F00400EFD70201376B90EC36F0A1C17D
:1069800064F1CFEC06F014D0A1C159F143EC05F04D
:1069900000090EE193EC37F0A1C15AF14CEC05F07F
:1069A0000101FE0EA16F0101090EA76F010E02D0B9
:1069B000000E00D012000B01006B070EE76E0019ED
:1069C000E8AE02D0E73402D0E750005D2CE2040EBE
:1069D000E66EE66A00CBE9FFEA6AE9BEEA68D890AB
:1069E000E936EA36260EE926030EEA22EECF10F04B
:1069F000EFCF11F0126A10C0E6FF11C0E6FF12C01F
:106A0000E6FFE5C1E6FFE6C1E6FF47EC47F0136E9F
:106A1000070EE15E1350000903E10B010051120063
:106A20000B01002BCAD7070C0B01036BB10E006FD3
:106A3000010E016F47D8EF50200804E1002B000E33
:106A40000123F8D700CBD3F101CBD4F10101010E22
:106A5000E16F38D8EFCF02FBEF5033E00B01035169
:106A6000010A16E0010A29E1200E025D03E02C0E66
:106A7000025D05E127D8EF6A010E036F1ED00D0EEF
:106A8000025D03E00A0E025D18E11CD8EF6A15D022
:106A9000200E025D12E00101E151E12BE96EEA6A8C
:106AA000D890E936EA36D30EE926010EEA2200CB69
:106AB000EEFF01CBEDFF0B01036B002B000E01235A
:106AC000C8D7120000CBE9FF01CBEAFF1200CCC30C
:086AD000E2F1CDC3E3F1120075
:086AD8000201306B010E316F69
:106AE0000301180E956F56EC45F00B01006B060E76
:106AF000005D05E2005125DAEF6A002BF8D7010CA2
:106B00000B01FE0E026F020131B102D0FE0EFFD06A
:106B10000B01016B060E0B01015D14E20B0101512B
:106B2000080DF3CFE9FFF4CFEAFF000EE926020ECD
:106B3000EA22EF50010B03E101CB02FB03D00B0172
:106B4000012BE8D7FE0E0B01025D02E1FE0EDFD045
:106B50000B01450E036F046B056B33C2E9FF34C2B2
:106B6000EAFFEF5002E1FF0ED2D033C2E6FF34C29B
:106B7000E6FF1CEC48F0E552E552F3CF33F2F4CFD8
:106B800034F203CB9AF304CB9BF30301A00E996F6D
:106B900095EC45F0000904E00B01FE0E026FB2D047
:106BA000E0EC45F00B01006F0B0100AF03D00B01CF
:106BB0000269A8D00B01016B0C0E0B01015D2AE2EA
:106BC000E0EC45F00B01006F0B0101510201EA6A94
:106BD0003325E96E3451EA22EF500B01005D0AE0E3
:106BE000120E0B010327000E0B010423000E0B01F4
:106BF000052310D00B0100510AE10B01012B0C0EF3
:106C00000B01015D03E2E0EC45F0F7D703D00B0187
:106C1000012BD2D70C0E0B01015D70E10B0102516B
:106C2000080DF3CF06FBF4CF07FB000E0B01062780
:106C3000020E0B01072306CBE9FF07CBEAFF010E8B
:106C4000EF6E06CBE9FF07CBEAFF010EEB6A020EFF
:106C5000EB6AE0EC45F0E66E06CBE9FF07CBEAFF16
:106C6000030EE926000EEA22E552E750EF6EE0EC53
:106C700045F0E66E06CBE9FF07CBEAFF030EE926F7
:106C8000000EEA22010EE926000EEA22E552E75044
:106C9000EF6EE0EC45F0E66E06CBE9FF07CBEAFFCE
:106CA000030EE926000EEA22020EE926000EEA2271
:106CB000E552E750EF6EE0EC45F0E66E06CBE9FFFB
:106CC00007CBEAFF060EE926000EEA22E552E7505E
:106CD000EF6EE0EC45F0E66E06CBE9FF07CBEAFF8E
:106CE000060EE926000EEA22010EE926000EEA222F
:106CF000E552E750EF6E0201302B04D0EAEC45F08C
:106D000004003FD7EAEC45F00B01025100D012001D
:106D100036C237F205D80201365113D9EF6A120094
:106D200002013751080DF3CFA4FBF4CFA5FB000EF1
:106D30000B01A427020E0B01A523A4CBE9FFA5CBD1
:106D4000EAFFEF50020B03E0EAEC45F012D0A4CBCF
:106D5000E9FFA5CBEAFFEF50040B0BE0D6EC45F0C2
:106D60000301A00EA36F25EC46F0000902E0040029
:106D7000F7D7F90E106EA4CBE9FFA5CBEAFF1050B0
:106D8000EF1602013193120002013851080DF3CFC2
:106D900001FBF4CF02FB000E0B010127020E0223C0
:106DA0009F0E106EC4D8E850EF16C1D8EF50010BFB
:106DB0001BE0BDD8EF50020B1AE1020131B314D031
:106DC000B6D8ECD8B4D8C7D810C09AF311C09BF38A
:106DD0000301A00E996F95EC45F0000905E1A7D8D5
:106DE000EF820201318303D0A2D8EF8A000CE0ECDD
:106DF00045F00B01006F9BD8C8D899D8BAD805E1E7
:106E00001350111802E193D8EF8C0B0100511200BE
:106E1000010C02013951080DF3CF00FBF4CF01FB47
:106E2000000E0B010027020E012386D8EF50040B41
:106E300005E0400E0201325D01E3BED87DD8EF507F
:106E4000040B16E1020131A303D076D8EF8A000CBF
:106E500073D8A4D871D87FD810C097F311C098F315
:106E6000A4D805E169D8EF840201318301D0000C78
:106E70003AC29CF3C2EC45F05FD887D85DD879D888
:106E800005E11350111802E157D8EF8C010C1200E4
:106E90001200F36AF46A1200056A066A076A1200B1
:106EA000000C020131A1000C0B01A46B060EA45DC5
:106EB00008E2A45146D8EF50010B01E0000CA42BCE
:106EC000F5D70201010E006F400E036F046B056BD6
:106ED000010C0B01000EA66F020EA76F020100A5A8
:106EE00004D0400E325D01E367D8020100B510D036
:106EF00031A302D0008B000C03C297F304C298F3B5
:106F000054D805E1020100853183326B01D0000CB9
:106F100045C29CF3C2EC45F00201322B032B000E5C
:106F200004230523010C48D80201006B010C01CB9E
:106F3000E9FF02CBEAFF120000CBE9FF01CBEAFF39
:106F40001200080DF3CFE9FFF4CFEAFF000EE926A7
:106F5000020EEA221200030EE926000EEA22EE508B
:106F60001324106EEE501420116EEE501520126E88
:106F70001200060EE926000EEA22EECF12F0EFCF45
:106F800013F00001125010181200EE52EE2A000EFB
:106F9000ED22EECF10F0EDCF11F01200EE52EECF59
:106FA00013F0EFCF14F0156A12000301A00E966FD4
:106FB0005FEC45F0000912000201376B90EF36F0EC
:106FC000AA6AA96A3F0EA6160B01D10E006F000E29
:106FD000016FA950106E116A120E105C000E11584C
:106FE0000CE2A68000CBE9FF01CBEAFF002B000EEC
:106FF0000123A8CFEFFFA92AECD71200EFC0A9FF09
:10700000AA6AA6A202D00400FCD73F0EA616A6804C
:10701000A85000D01200A8CF5DFBF0C0A9FFAA6A5B
:10702000A6A202D00400FCD73F0EA616A6800B0134
:107030005D51A85C01E111D05DCBA8FF2F0EA61613
:10704000A684550EA76EAA0EA76EA6820000A6A261
:1070500002D00400FCD7A69400D012001200240E27
:10706000AC6E900EAB6E080E7E6E00011F0ECED978
:10707000080A36E00F0A32E0010A2AE0030A23E098
:10708000010A1CE0070A15E0010A0EE0030A07E006
:10709000010A28E10B01340E486F820E1DD00B014E
:1070A0008C0E486F200E18D00B01450E486F100E45
:1070B00013D00B01220E486F080E0ED00B01100EDC
:1070C000486F040E09D00B01080E486F020E04D061
:1070D0000B01030E486F010E496F08D0AC0E03D0B0
:1070E000560E01D0AC0E0B01486F496B48CBAFFF79
:1070F00049CB10F0116A10507F6E12000001230E70
:1071000085D9926E0001240E81D9936E0001250E5F
:107110007DD9D809946E0001280E78D9976E0001A8
:10712000290E74D91009986E120000012A0E6ED92A
:10713000896E00012B0E6AD98A6E00012C0E66D969
:107140008B6E00012F0E62D98E6E0001300E5ED95B
:107150008F6E12000001310E59D9C16E0001320E3E
:1071600055D97F0BC06E1200010E0001F15D4AE39C
:10717000F151050801E21200F45111E0F2C0A8FF3C
:10718000F105E824660F0001F06F45DFF3C0A8FFAA
:107190000001F105E824670F0001F06F3CDF0001FA
:1071A000F10526D9EECF58FBEDCF59FB58CB5AFB52
:1071B00059CB5BFB0B01010E5A5F000E5B5B060EA9
:1071C0000001D890F237F337E806FBE10001F251F5
:1071D000E840E8403F0B300B106E5ACBE9FF5BCB29
:1071E000EAFFEF50CF0B10100B015C6F58CBE9FF9B
:1071F00059CBEAFFF3C0EFFF5ACBE9FF5BCBEAFFC5
:107200005CCBEFFF12000B01106B116B010E000144
:10721000F55D2DE3F551050801E21200F505E8D80A
:10722000EECF0CFBEDCF0DFB0CCB0EFB0DCB0FFB14
:107230000B01010E0E5F000E0F5B0CCBE9FF0DCBB7
:10724000EAFFEF50106F116BD89010371137D890BC
:10725000103711370ECBE9FF0FCBEAFFEF50300BA1
:10726000E8380F0B101310CBF3FF11CBF4FF120013
:10727000F6C058FB0001F75106E058CBA8FF00010B
:10728000640EF06FC8DECB50106E116AFF0E10183E
:1072900001E1115002E0000E01D0010E010808E1E9
:1072A000030E0B01585D02E1586B0BD0020E06D0A5
:1072B0000B01585102E1020E03D0030ED88058553D
:1072C000586F030E5817FC0ECA165851CA121200F6
:1072D000030ECA140B010C6F030E0C5D01E10C07C9
:1072E000CB50106E116AFF0E101804E1115002E12C
:1072F000020E01D0030ED8800C5512000001F95186
:1073000006E0F8C0A8FF0001630EF06F84DE000104
:10731000F8A103D00C0EBD1202D0F00EBD16F8A3DA
:1073200003D00C0EBA1202D0F00EBA16F8A504D093
:107330000C0EB7123C0E01D0F00EB716F8A704D011
:107340000C0E73123C0E01D0F00E7316F85102E0D1
:10735000CA841200CA9412000001630E57D80009B3
:1073600001E11200B70EB1160001650E4FD8010BF6
:1073700002E0CB6802D03F0ECB6E0001F76B00013C
:10738000640E44D80001F66F73DF0001660E2BD83F
:10739000670E1ED8010E36D8680E25D8690E18D88B
:1073A000020E30D86A0E1FD86B0E12D8030E2AD8E0
:1073B0006C0E19D86D0E0CD8040EF16FD5DE0001DD
:1073C000F96B0001630E22D80001F86F7EEF39F0EF
:1073D0001DD80B01496F0001F46B48CBF2F0E8CFE8
:1073E000F3F00001120012D80B01486F00011200E7
:1073F000E96EEA6AD890E936EA36B90EE926030E54
:10740000EA221200F16FB0DE00011200EF6FFEEF12
:0274100037F053
:0E7412000201FF51020A1EE0030A06E0010A11
:1074200001E048D10201FF2B45D1890E0001B56F63
:10743000B66B0001B36BB46B890E0001B16FB26B18
:10744000EFEC25F00D01FB6FFF0E0D01FB5D01E17F
:1074500031D10201FF2BFBCDBEF06FEC27F000090C
:1074600001E128D10001060EBF6F0B0EC06F7EEC4C
:1074700027F00001050EBF6F0B0EC06F7EEC27F0EA
:107480000001080EBF6F0B0EC06F7EEC27F00001ED
:10749000070EBF6F0B0EC06F7EEC27F000010A0EC7
:1074A000BF6F0B0EC06F7EEC27F00001090EBF6F9F
:1074B0000B0EC06F7EEC27F000010C0EBF6F0B0EA1
:1074C000C06F7EEC27F000010B0EBF6F0B0EC06F7C
:1074D0007EEC27F000010E0EBF6F0B0EC06F7EEC2E
:1074E00027F000010D0EBF6F0B0EC06F7EEC27F072
:1074F0000001100EBF6F0B0EC06F7EEC27F0000175
:107500000F0EBF6F0B0EC06F7EEC27F00B0109CB87
:1075100010F00ACB11F00907000E0A5B1050111091
:1075200001E1C5D00D01110EFC6F0B0EFD6FEBD804
:107530000001000EBF6F0B0EC06F7EEC27F0000144
:10754000020EBF6F0B0EC06F7EEC27F00001010E24
:10755000BF6F0B0EC06F7EEC27F00001040EBF6FF3
:107560000B0EC06F7EEC27F00001030EBF6F0B0EF9
:10757000C06F7EEC27F00B01200E011901E10251D2
:1075800001E094D00B01010E031901E1045101E067
:107590008DD00D01110EFE6F0B0EFF6FE1D80009AB
:1075A00001E184D0FBCDB8F04FEC26F0000902E1F8
:1075B0000400F8D70B01076B840E086F06CBB9F0F7
:1075C0005BEC26F005CBB9F05BEC26F008CBB9F00C
:1075D0005BEC26F007CBB9F05BEC26F00001B96B51
:1075E0005BEC26F00001B96B5BEC26F00001B96B97
:1075F0005BEC26F00001010EB96F5BEC26F0000198
:10760000B96B5BEC26F00001B96B5BEC26F0000176
:10761000B96B5BEC26F00001B96B5BEC26F04BD844
:107620000001B96B5BEC26F00001200EB96F5BEC3A
:1076300026F00001B96B5BEC26F00001010EB96F7A
:107640005BEC26F00001B96B5BEC26F00001B96B36
:107650005BEC26F00001B96B5BEC26F00001B96B26
:107660005BEC26F00001B96B5BEC26F00001060E26
:10767000B96F5BEC26F00001600EB96F5BEC26F091
:107680000001B96B5BEC26F0D1C0B9F05BEC26F0E1
:10769000D2C0B9F05BEC26F0D3C0B9F05BEC26F0B9
:1076A000D4C0B9F05BEC26F0D8EC26F02FD7CCECA8
:1076B00027F000D012000001200EB96F5BEC26F01D
:1076C0000B01486B100E485D1AE2470E4825000179
:1076D000EF6FFEEC37F00B01496FE8380F0B410FED
:1076E0000001B96F5BEC26F00F0E0B014915410F3D
:1076F0000001B96F5BEC26F00B01482BE3D70001CA
:10770000B96B5BEF26F00001210EBF6F0B0EC06F4F
:107710007EEC27F00B0121512107000918E043D826
:107720002239F00B236F21073ED821511E08F2E3C6
:1077300023512211E66E0D01FCCDE9FFFDCDEAFFDC
:10774000FC2B000EFD23E552E750EF6EE3D70F0E42
:107750000D01EA6AFC25E96EFD51EA22EF6A12008A
:107760000B01216B0F0E215D1DE2470E212500014B
:10777000EF6FFEEC37F00B01226F0D01FECDE9FF3C
:10778000FFCDEAFFFE2B000EFF23EFCF23FB0B0103
:107790002351225D01E0000C2351225D01E0010C28
:1077A000212BE0D7010C0001220EBF6F0B0EC06F22
:0C77B0007EEC27F0410E0B01225F12005E
:0477BC00436163685A
:1077C000652D436F6E74726F6C3A206D61782D6118
:1077D00067653D3630302C206D7573742D7265767B
:1077E000616C69646174650D0A00485454502F310E
:1077F0002E302034303120556E617574686F726997
:107800007A65640D0A5757572D41757468656E7413
:1078100069636174653A20426173696320726561CE
:107820006C6D3D2264656661756C74220D0A0D0AEB
:1078300041757468656E7469636174696F6E205216
:1078400065717569726564210D0A00485454502FA2
:10785000312E3020353033200D0A0D0A53657276F3
:1078600069636520556E617661696C61626C650D56
:107870000A00485454502F312E3020343034204EDA
:107880006F7420666F756E640D0A0D0A4E6F74205A
:10789000666F756E642E0D0A00617564696F2F78CE
:1078A0002D77617665006170706C69636174696FD2
:1078B0006E2F6A6176612D61726368697665006911
:1078C0006D6167652F6A70656700696D6167652F17
:1078D00067696600746578742F6A61766173637294
:1078E00069707400746578742F63737300617070CD
:1078F0006C69636174696F6E2F6A6176612D766D54
:1079000000746578742F68746D6C00746578742FDA
:10791000706C61696E00477565737400596573001A
:107920000D0A4E6F772072756E6E696E67206170FA
:10793000706C69636174696F6E2E2E2E000D0A5291
:107940006561647920746F20646F776E6C6F616419
:107950002046696C652053797374656D20496D61AB
:107960006765202D2055736520586D6F64656D2007
:1079700070726F746F636F6C2E0D0A000D0A4448AD
:107980004350202620495020476C65616E696E6720
:107990002064697361626C65642E0D0A000D0A44EF
:1079A000484350202620495020476C65616E696E1F
:1079B0006720656E61626C65642E0D0A000D0A44D5
:1079C000656661756C74205375626E6574204D61D7
:1079D000736B2028000D0A44656661756C7420473E
:1079E00061746577617920416464726573732028DE
:1079F000000D0A44656661756C742049502041642D
:107A000064726573732028000D0A53657269616C96
:107A1000204E756D626572202800323030204F6B29
:107A20000D0A003432352043616E2774206372657D
:107A3000617465206461746120736F636B65742E7B
:107A40002020496E637265617365204D41585F5314
:107A50004F434B4554532E0D0A0032323620547298
:107A6000616E7366657220436F6D706C6574650D31
:107A70000A0031323520446F6E650D0A0031353011
:107A8000205472616E7366657272696E67206461FC
:107A900074612E2E2E0D0A00353330204C6F67692D
:107AA0006E2072657175697265640D0A0035303239
:107AB000204E6F7420696D706C656D656E746564C1
:107AC0000D0A00353030200D0A0032323120427963
:107AD000650D0A00323330204C6F6767656420699A
:107AE0006E0D0A003333312050617373776F726407
:107AF0002072657175697265640D0A00323230203A
:107B000052656164790D0A0041424F520054595048
:107B10004500504F52540053544F52005155495450
:0B7B20000050415353005553455200E4
:017B2B000059
:047B2C00DACFE4FFC9
:107B3000E2CFDAFFE9CFE4FFEACFE4FFF6CFE4FFDC
:107B4000F7CFE4FFF5CFE4FFF3CFE4FFF4CFE4FF9A
:107B5000FACFE4FF00EE00F0100EE80403E3EECFEE
:107B6000E4FFFBD700EE10F0100EE80403E3EECFC5
:107B7000E4FFFBD7E652F2A414D09E0ED76E580E47
:107B8000D66E0301CC2B000ECD23CE23CF230301D1
:107B9000D20706E1640ED26F0301D02B000ED12371
:107BA000F2949E50200B05E09D50200B02E045EC26
:107BB00048F09E50100B05E09D50100B02E05BEC6E
:107BC00048F0E55200EE1FF0100EE80403E3E5CFA5
:107BD000EDFFFBD700EE0FF0100EE80403E3E5CF56
:107BE000EDFFFBD7E5CFFAFFE5CFF4FFE5CFF3FFDD
:107BF000E5CFF5FFE5CFF7FFE5CFF6FFE5CFEAFFED
:107C0000E5CFE9FFE5CFDAFF1100040012001ED92D
:107C1000C5EC4AF06CEC35F09FEC29F031EC48F003
:107C2000E0EC37F02FEC38F03AEC48F07EEC38F02E
:107C300095EC38F0AAEC38F0ACEC39F00001140EF9
:107C4000EF6FFEEC37F00F01526F0DEC2DF0F7ECFB
:107C500041F02AEC10F0F1EC32F0A4EC16F0BDEC9F
:107C600021F00001160EEF6FFEEC37F0010B06E17C
:107C70000F01010E5D6F0301080ED76FCF6ACE6A48
:107C80000001150EEF6FFEEC37F0020B0CE00F0158
:107C90005E510301CC5D106E320E105C04E3CCC368
:107CA0005EFF939C8A7C0F015F510301CC5D106ED7
:107CB000010E105C02E3CCC35FFF02EC42F0DAEC91
:107CC00016F063EC10F000EC33F009EC3AF008D851
:107CD0000F015D510301DA5DD1E0DAC35DFFCED75C
:107CE0000301A42B0C0E0301A45D02E30301A46BAA
:107CF000C11C0F0B0301A45D17E2C30EC2160301E2
:107D0000A451040DF350C212C280C282C2A202D09A
:107D10000400FCD70301A451EA6AE30FE96E000EE8
:107D2000EA22C4CFEFFF08D00301A451EA6AE30FAF
:107D3000E96E000EEA22EF6A12000201D20ECC6F49
:107D4000950ECD6FA7C3CAF2A8C3CBF2EBEC31F00E
:107D5000000961E00201080EC56F350E0201C36F14
:107D6000C46B0201880EC16F0B0EC26F9AEC31F02A
:107D70000B01876FE850872BEA6A880FE96E0B0EBC
:107D8000EA223A0EEF6E0201080EC56F3E0E0201A6
:107D9000C36FC46B0B0187510201C16FC26B880EA8
:107DA000C1270B0EC2239AEC31F0880EE66E0B0E43
:107DB000E66EE0EC47F0E552E552F3CFDBF202016C
:107DC000880ED96F0B0EDA6F02019C0ED76F0B0E67
:107DD000D86F34EC32F09C0EE66E0B0EE66E150E8C
:107DE0000301116AA725106EA851112210C0E6FFE9
:107DF00011C0E6FF91EC47F0E552E552E552E5523D
:107E0000000909E1A5C3E9FFA6C3EAFF090EE926B7
:107E1000000EEA22EF841200350E0201C86FC96B12
:107E2000ABC3C6F2ACC3C7F2CCEC31F000090DE134
:107E30003E0E0201C86FC96BADC3C6F2AEC3C7F236
:107E4000CCEC31F0000901E1010C000C810ECD6E8B
:0A7E5000F18ED56AF28EF28C12005A
:067E5A00140E02018F6FFF
:107E6000906B0201020E8D6F0B0E8E6FA1EC1EF057
:107E7000F00E0B010215400801E0000C0F0E021578
:107E8000040DF3CF62F3F350106E116A140E105EFE
:107E9000000E115A10C01CFB1050280801E2000C03
:107EA0001C5100080BE21C5102018F6F906B020104
:107EB0001D0E8D6F0B0E8E6FA1EC1EF00CCB16FB02
:107EC0000DCB17FB0B010C6B0D6B140E1BD9020EA7
:107ED000B16F0B0EB26F53EC30F0F3CF18FBF4CF51
:107EE00019FB0B01181F191F1C51000810E21C512F
:107EF00009D91D0EB16F0B0EB26F53EC30F0F3CFFA
:107F00001AFBF4CF1BFB0B011A1F1B1F02D01A6BAD
:107F10001B6B040EF7D8180EB16F0B0EB26F53EC3B
:107F200030F0F3CF00FBF4CF01FB0B01F350161937
:107F300002E10151171901E0000C0301020E726FFA
:107F40000B0E736FB2D80301635164110CE063C36D
:107F5000E9FF64C3EAFF12CBEEFF13CBEEFF14CBB5
:107F6000EEFF15CBEEFF65C3E9FF66C3EAFF060E21
:107F7000E3D80ECBEEFF0FCBEEFF10CBEEFF11CB15
:107F8000EEFF67C3E9FF68C3EAFF0BCBEFFF625167
:107F9000126E136A0B011250045D106E13500559D6
:107FA000116E69C3E9FF6AC3EAFF10C0EEFF11C09A
:107FB000EDFF010C0301140E626F0B01450E2B6FD8
:107FC0002C6B140E03016E250B012D6F000E0301A7
:107FD0006F210B012E6F0301DF2B000EE023DFC3A7
:107FE0002FFBE0C330FB0B01316B400E326F640E90
:107FF000336F6DC334FB356B366BD1C037FBD2C0EA
:1080000038FBD3C039FBD4C03AFB6BC3E9FF6CC368
:10801000EAFF060E91D8EECF3BFBEECF3CFBEECF56
:108020003DFBEFCF3EFB03012B0E726F0B0E736F08
:108030003CD8140E67D82B0EB16F0B0EB26F53ECF9
:1080400030F0F3CF35FBF4CF36FB140E03016E2571
:1080500002019E6F000E03016F2102019F6F02015A
:108060009D6B6BC3E9FF6CC3EAFF6BC39BF26CC3F0
:108070009CF261EC20F0140E02018B6F8C6B0201FC
:108080002B0E896F0B0E8A6FE9EC1DF0F36AF46A10
:1080900012000301625170250201A56F000E030159
:1080A00071210201A66F1CEF21F027D8020E35D8EE
:1080B000020E38D8020E2BD8020E39D8040E2DD855
:1080C000040E30D8040E23D8040E31D8060E25D85D
:1080D000060E28D8060E1BD8060E29D80A0E1DD863
:1080E0000A0E20D80A0E13D80A0E03D845CBEFFF8C
:1080F000120022D8010E9CEF40F072C3E9FF73C357
:10810000EAFF12000201B36FB46B0201120014D82F
:10811000E552E750EF6E7DEF40F00ED8EFCF45FB14
:108120007DEF40F0E6DFEF50E66E7DEF40F0E1DFFF
:1081300045CBEFFF7DEF40F0E926000EEA2212006A
:108140001C0E02018F6F906B0201000E8D6F0B0EE3
:108150008E6FA1EC1EF06CEC1FF00301000ECA6FD5
:108160000B0ECB6F08D90B01010E001912E1015162
:1081700010E10451106E116A060E10180AE1115038
:1081800008E10551126E136A040E121801E1135032
:1081900001E0000C020E061905E1075103E119D9AF
:1081A000EF6A0DD0010E061906E1075104E1010E38
:1081B00010D9EF6E04D0020E0CD9EF6E000C000146
:1081C000D1510B01185D2EE10001D2510B01195D57
:1081D00029E10001D3510B011A5D24E10001D451C2
:1081E0000B011B5D1FE1C3C3E9FFC4C3EAFF08CB5A
:1081F000EEFF09CBEEFF0ACBEEFF0BCBEEFF0CCB75
:10820000EEFF0DCBEEFFC3C3E9FFC4C3EAFF060ECA
:10821000EAD80ECBEEFF0FCBEEFF10CBEEFF11CB6B
:10822000EEFF010C000C0201010E876FAFEC1DF098
:108230000B011C6FFF0E1C5D01E1000C0201A86B1D
:10824000A96B1CCBA7F22FEC21F0010E0B01006FE4
:10825000016B026B080E036F060E046F040E056FB0
:108260000301C9050BE1010E0B01066F076B1269D3
:108270001369146915691669176914D0020E0B0188
:10828000066F076BC7C3E9FFC8C3EAFFEECF12FB57
:10829000EECF13FBEECF14FBEECF15FBEECF16FBAC
:1082A000EFCF17FBD5C008FBD6C009FBD7C00AFB30
:1082B000D8C00BFBD9C00CFBDAC00DFBD1C00EFB44
:1082C000D2C00FFBD3C010FBD4C011FB7BD8EF5042
:1082D0000E190001DB151BE175D8010E84D8EF5093
:1082E0000B010F190001DC1512E16CD8020E7BD8CE
:1082F000EF500B0110190001DD1509E163D8030EE1
:1083000072D8EF500B0111190001DE1509E0DFC032
:1083100018FBE0C019FBE1C01AFBE2C01BFB09D04F
:1083200051D8EECF18FBEECF19FBEECF1AFBEFCFF3
:108330001BFB0301000ECA6F0B0ECB6F1CD81C0E6B
:1083400002019E6F9F6B0201060E9D6F0201120ECD
:108350009B6F0B0E9C6F61EC20F01C0E02018B6F6B
:108360008C6B0201000E896F0B0E8A6FE9EC1DF019
:10837000B9EC20F0010C32D819D8F3CFEEFF11C0C0
:10838000EDFF2CD8020E2FD811D8020EF3CFEBFF41
:10839000030E11C0EBFF22D8060E25D807D8060E13
:1083A000F3CFEBFF070E11C0EBFF1200EECFABF2E5
:1083B000EDCFACF21FEC30F0F3CF10F0F4CF11F0B2
:1083C000EEEF41F0C7C3E9FFC8C3EAFF060EF3EFC3
:1083D00041F0C5C3E9FFC6C3EAFF1200CAC3E9FF03
:0E83E000CBC3EAFF1200E926000EEA221200CB
:0283EE0002018A
:1083F000476B4681AEEC1CF0F5EC48F0E3EC25F061
:1084000058EF04F00B01B26B02014751040A01E17D
:10841000EFD0070A01E1B9D0050A01E1A1D0010AB4
:1084200001E189D0050A49E0070A40E0050A03E0B6
:10843000010A01E0FFD00201B10E996F0B0E9A6F95
:108440000201480E976F020E986FB1EC1FF0000901
:1084500018E10001160EEF6FFEEC37F0010B10E093
:10846000A3EC1FF000090CE10001D16B0001D26BFD
:108470000001D36B0001D46B02014681BDEC21F0F9
:10848000D9D00B01010EB26F0B01B15104E1020111
:10849000020E476F0AD0060E0B01B15D04E1020126
:1084A000050E476F02D06CEC1FF0C4D002EC49F00F
:1084B000000902E00201476BBDD00301520E696F53
:1084C000020E6A6F0301B10E676F0B0E686F030136
:1084D000480E656F020E666F0301AD0E636F0B0EE3
:1084E000646F2DEC3FF0000921E00B01010EB26F2B
:1084F0000B01B10504E10201030E476F16D0060E11
:108500000B01B15D04E10201060E476F0ED0110EA2
:108510000B01B15D04E10201070E476F06D00B01AC
:10852000B26B6CEC1FF00201476B04D06CEC1FF0D7
:108530000201476B7FD052C2C9F053C2CAF000019A
:10854000AD0EC76F0B0EC86F0001480EC56F020E4F
:10855000C66FD4EC27F0000902E00201476B6AD035
:1085600052C277F153C278F10101AD0E756F0B0E57
:10857000766F0101480E736F020E746F09EC09F0FB
:10858000000902E00201476B55D00201476B02016E
:10859000290ED8805255000E535527E30301760E5D
:1085A000546F020E556F0301740E526F020E536F1B
:1085B0000301520E506F020E516F0301540E4E6FA5
:1085C000020E4F6F0301B10E4C6F0B0E4D6F2BEC73
:1085D00043F000090AE0080E0B01B15D06E10B0152
:1085E000010EB26F0201040E476F6CEC1FF022D037
:1085F0000201010E866F93EC1DF000091AE076C2AD
:108600005EF377C25FF374C25CF375C25DF352C26E
:108610005BF30301540E596F020E5A6F0301586B3E
:108620000301480E566F020E576FA5EC43F002018E
:10863000476B00D004000B01B25101E0E3D6EEEC31
:1086400007F0D0EC21F00301D9A102D0020146913C
:068650007AEC1DF012009F
:0A865600080E02018F6F906B020105
:10866000000E8D6F0B0E8E6FA1EC1EF0080E106EBB
:1086700004D9E850EF5E01D9EF5002018F6F906B83
:108680004EC38DF24FC38EF2A1EC1EF002CB2AFB3B
:1086900003CB2BFB0B01026B036B080E0201B36FC4
:1086A000B46B0201000EB16F0B0EB26F53EC30F0E1
:1086B000F3CF2CFBF4CF2DFB0B012C1F2D1FDDD88E
:1086C000EF500201B36FB46B4EC3B1F24FC3B2F2BD
:1086D00053EC30F0F3CF2EFBF4CF2FFB0B012E1F0A
:1086E0002F1F040E0201B36FB46B02012C0EB16F89
:1086F0000B0EB26F53EC30F0F3CF28FBF4CF29FB15
:108700000301000E606F0B0E616F8CD84CC3E9FF44
:108710004DC3EAFF00CBEFFF52C3E9FF53C3EAFFAB
:1087200004CBEEFF05CBEDFF54C3E9FF55C3EAFFD1
:1087300006CBEEFF07CBEDFF0B012A51281902E112
:108740002B51291901E0000C010C0201010E876F69
:10875000AFEC1DF00B012A6FFF0E2A5D01E1120044
:10876000140E0201A86FA96B2ACBA7F22FEC21F0FF
:10877000080E03015B250B01286F296B000E2923CE
:10878000016B58C300FB026B036B5CC304FB5DC34E
:1087900005FB5EC306FB5FC307FB03015B51E66E8F
:1087A000E66A59C3E6FF5AC3E6FF080EE66E0B0EF3
:1087B000E66E66EC47F0106E060EE15E10500301A7
:1087C000000E606F0B0E616F2DD828CBB3F229CB52
:1087D000B4F20201000EB16F0B0EB26F53EC30F029
:1087E000F3CF02FBF4CF03FB080E03015B2503016B
:1087F0006E6F6F6B000E6F230301010E6D6F56C31A
:108800006BF357C36CF3DAEC3FF028CB8BF229CB38
:108810008CF20201000E896F0B0E8A6FE9EC1DF0DD
:10882000B9EF20F02FD8040E15D8040EF3CFEBFFCC
:10883000050E1FD8060E0ED8060EF3CFEBFF070E5F
:1088400018D8020E07D8020EF3CFEBFF030E11C0AB
:10885000EBFF1200E926000EEA22EECFABF2EDCFDD
:10886000ACF21FEC30F0F3CF10F0F4CF11F042EF88
:1088700044F011C0EBFF42EF44F050C3E9FF51C395
:0E888000EAFF120060C3E9FF61C3EAFF1200C5
:02888E00FF0EDB
:10889000E3CFEAFFE552FF0EE3CFE9FFE552E66AD8
:1088A000E66AD9CFE6FFDACFE6FFFC0EE124D96E07
:1088B000FF0EE220DA6EE66AE66AE66A200EEF5CF8
:1088C00006E0090EEF5C03E0EF6603D03FD0EE5008
:1088D000F5D72D0EEF5C03E1FF0EE32A03D02B0E3C
:1088E000EF5C01E1EE502F0EEF6424D03A0EEF6002
:1088F00021D0D890F90EE336FA0EE336FD0EDECF26
:10890000E3FFFE0EDDCFE3FFD890F90EE336FA0E5B
:10891000E336D890F90EE336FA0EE336FD0EE35057
:10892000DE26FE0EE350DD22300EEE5CDE26000E6B
:10893000DD22D9D7FF0EE3CFE8FFE85207E0F90EBA
:10894000E31EE32AFA0ED8B4E306E31EE552E5522D
:10895000E552FF0EE3CFDAFFE552FF0EE3CFD9FF7A
:10896000E552E1CFE9FFE2CFEAFFED52ED52EECF63
:10897000F3FFEFCFF4FF1200D9CFE6FFDACFE6FF27
:10898000FA0EE3CFD9FFFB0EE3CFDAFFFD0EE35281
:1089900009E72D0EDE6EFC0EE31EE32AFD0ED8B4B1
:1089A000E306E31EE652E652E652FD0EE124E76ED0
:1089B000FF0EE220E46EE652F70EE3CFE6FFF70E7D
:1089C000E3CFE6FF2CEC45F0F90EE124E96EFF0E53
:1089D000E220EA6E1CEC45F00AE119EC45F009E1F1
:1089E0001CEC45F008E119EC45F007E108D027EC54
:1089F00045F022EC45F027EC45F022EC45F027EC61
:108A000045F0DE6AF90EE126FF0EE222FF0EE3CF0B
:108A1000DAFFE552FF0EE3CFD9FFE552FC0EE12469
:108A2000E96EFF0EE220EA6EEECFF3FFEFCFF4FF28
:108A30001200EF380F0B1200EF500F0B02E1EE5255
:108A4000D8841200EF380F0B300FDE6E1200EE509C
:108A50000F0B300FDE6E1200FC0EE3CFE9FFFD0EB0
:108A6000E3CFEAFF100EE66EEE6AEE6AEF6AD89088
:108A7000FD0EE336FE0EE336ED36ED36EF36FF0E35
:108A8000E30609E04DEC45F0EE524DEC45F0EE52B8
:108A90004DEC45F0EDD7E56E1200030EEF24E8B67D
:0C8AA000EF6E300EEF24E8BEEF6E000C0D
:048AAC0095C3D5F3A6
:108AB0000301D46B0301080ED36F61EF4AF097C333
:108AC000A4FB98C3A5FBC750040B01E0010EE5D839
:108AD000FAE1C580C5B0FED7A1B6010C96C3D6F3A6
:108AE000E1D801E0010CC750040B01E0010ED5D81C
:108AF000FAE1C5BC19D0A5CBD6F3D4D801E0010C5E
:108B0000C750040B01E0010EC8D8FAE1A4CBD6F39C
:108B1000C9D801E0010CC750040B01E0010EBDD81B
:108B2000FAE1C5AC000C020C020C9AC397F39BC38C
:108B300098F399C396F3C3DF0B01086FE85005E182
:108B400078D80B01086FE85002E008511200C750B6
:108B5000040B01E0010EA1D8FAE1C580C5B0FED733
:108B6000A1B6010C030199290301D66F9BD801E03E
:108B7000010CC750040B01E0010E8FD8FAE1C5AC1F
:108B8000000C020CC750040B01E0010E86D8FAE17C
:108B90009CC3D6F387D801E0010CC750040B01E059
:108BA000010E7BD8FAE1C5AC000C020CC750040BD7
:108BB00001E0010E72D8FAE1C584C5B4FED7000CFD
:108BC00070EC4AF0C5B6FED7C59AC588C5B8FED7C1
:108BD000C950120070EC4AF0C5B6FED7C58AC588E8
:108BE000C5B8FED7C584C5B4FED7000C9EC39AF3A2
:108BF0009FC39BF39DC399F398DF0B01006FE8506F
:108C000016E10301A251A20700090EE0D9DFE66ECA
:108C10000301A0C3E9FFA1C3EAFFA02B000EA1231B
:108C2000E552E750EF6EEDD7D5DF0B01006F005135
:108C30001200C750040B01E0010E2FD8FAE1C584E1
:108C4000C5B4FED7A1B6010C000CC750040B01E05F
:108C5000010E23D8FAE1C580C5B0FED7A1B6010C3C
:108C6000A3C3D6F31FD801E0010CC750040B01E0E9
:108C7000010E13D8FAE1A1B6010CC5BC03D00B015B
:108C8000A86B03D00B01040EA86FC584C5B4FED732
:108C9000A1B6010C0B01A8511200106E1F0EC514D5
:0C8CA0001010120075EC4AF000091200E0
:048CAC000D0A5072EB
:108CB00065737320616E79206B657920666F722011
:108CC000436F6E66696775726174696F6E206D655A
:108CD0006E752E000D0A52756E6E696E67204170BA
:108CE000706C69636174696F6E2C204950206164F7
:108CF00064726573733A2000444843502F476C6593
:108D0000616E696E672E2E2E000D0A0D0A0D4D6FD5
:108D10006474726F6E69782057656220536572764D
:108D200065720D0A0D0A09313A204368616E676564
:108D300020426F6172642073657269616C206E7588
:108D40006D6265722E0D0A09323A204368616E67C2
:108D5000652064656661756C7420495020616464A7
:108D6000726573732E0D0A09333A204368616E678A
:108D7000652064656661756C7420676174657761F0
:108D80007920616464726573732E0D0A09343A2088
:108D90004368616E67652064656661756C742073F5
:108DA00075626E6574206D61736B2E0D0A09353A1C
:108DB00020456E61626C652044484350202620495E
:108DC0005020476C65616E696E672E0D0A09363A50
:108DD0002044697361626C6520444843502026201A
:108DE000495020476C65616E696E672E0D0A093720
:108DF0003A20446F776E6C6F61642046696C652021
:108E000053797374656D20496D6167652E0D0A098C
:108E1000383A2053617665202620517569742E0DED
:108E20000A0D0A456E7465722061206D656E7520AD
:108E300063686F6963652028312D38293A20000D59
:108E40000A496E76616C696420696E70757420726F
:108E500065636569766564202D20496E70757420A0
:108E600069676E6F7265642E0D0A507265737320A8
:108E7000616E79206B657920746F20636F6E746901
:0E8E80006E75652E2E2E0D0A001B5B324A0009
:028E8E00FB0ED9
:108E9000E3CFF6FFFC0EE3CFF7FFFD0EE3CFF8FFC5
:108EA000FE0EE3CFE9FFFF0EE3CFEAFFF90EE3503A
:108EB00003E1FA0EE35009E0F90EE30602E2FA0ECE
:108EC000E3060900F550EE5CF1E01200D9CFE6FFB1
:108ED000DACFE6FFFA0EE3CFD9FFFB0EE3CFDAFFDE
:108EE000FC0EE3CFE9FFFD0EE3CFEAFFE9CFF3FF8E
:108EF000EACFF4FFF80EE35003E1F90EE35008E087
:108F0000F80EE30602E2F90EE306DECFEEFFF2D73B
:108F1000FF0EE3CFDAFFE552FF0EE3CFD9FFE552B4
:108F20001200D9CFE6FFDACFE6FFFA0EE3CFD9FF82
:108F3000FB0EE3CFDAFFFC0EE3CFE9FFFD0EE3CF3C
:108F4000EAFFDE50EF5C02E1EE66FBD7F36EFF0E48
:108F5000E3CFDAFFE552FF0EE3CFD9FFE552F3503E
:108F60001200FB0EE3CFF6FFFC0EE3CFF7FFFD0E82
:108F7000E3CFF8FFFE0EE3CFE9FFFF0EE3CFEAFFFA
:108F80000900F550EF5C02E1EE66FAD71200FB0E25
:108F9000E3CFF6FFFC0EE3CFF7FFFD0EE3CFF8FFC4
:108FA000FE0EE3CFE9FFFF0EE3CFEAFFE9CFF3FFC9
:108FB000EACFF4FF0900F5CFEFFFEE66FBD7120012
:108FC000FE0EE3CFE9FFFF0EE3CFEAFFF36AF46A98
:108FD000EE5203E0F34AF42AFBD71200D9CFE6FFA2
:108FE000DACFE6FFFA0EE3CFD9FFFB0EE3CFDAFFCD
:108FF000FC0EE3CFE9FFFD0EE3CFEAFFE9CFF3FF7D
:10900000EACFF4FFF80EE35003E1F90EE3500BE072
:10901000F80EE30602E2F90EE306DECFEFFFEE669E
:10902000F1D7DD52EFD7FF0EE3CFDAFFE552FF0EA7
:10903000E3CFD9FFE5521200FE0EE3CFE9FFFF0EAA
:10904000E3CFEAFFE9CFF3FFEACFF4FF610EEF5C75
:1090500005E67B0EEF5C02E7DF0EEF16EE52F6E15F
:029060001200FC
:0E9062000D01F46BE86BE96BF26BF36B9D9AFA
:109070009D9812009D8A9D9812000D01E96BE9CD23
:10908000E8FDF36BF3CDF2FD1200060EAB1402E027
:10909000AB98AB889EAA0ED00D01F351EA6AEA0F95
:1090A000E96E0D0EEA22AECFEFFFF32B070EF3159C
:1090B000F36FF0D712000D01E851E95D0DE0E851C2
:1090C000EA6A680FE96E0D0EEA22EF50AD6EE82BEA
:1090D0007F0EE815E86F12009D98120012000D0136
:1090E000F45112000D01F251EA6AEA0FE96E0D0E19
:1090F000EA22EFCFA4FBF22B070EF215F26F0B0161
:10910000A45112000D01E929106E116A7F0E10168C
:10911000000E11160D01E851126E136A125010184C
:1091200002E11350111802E10400ECD7F29E9DB841
:1091300005D0F5CDADFF9D88F28E11D00D01E9511E
:10914000EA6A680FE96E0D0EEA22F5CDEFFF0D0118
:10915000E92B7F0E0D01E9150D01E96FF28E12006A
:109160000D01F6519F0805E2F6390F0B0F0B570F53
:1091700004D0F6390F0B0F0B300F0D01F56FC2DF66
:109180000F0E0D01F615090804E20F0EF615570F24
:1091900003D00F0EF615300F0D01F56F82EF48F07A
:1091A0000D01F7CDE9FFF8CDEAFFF72B000EF8230C
:1091B000EFCF08FBEF5005E008CBF5FDA3DF04007F
:1091C000EFD712000D01F9CDF6FFFACDF7FFF92B1D
:1091D000000EFA230800F5CF00FBF55005E000CBA8
:0A91E000F5FD90DF0400EED7120049
:0691EA000301746B7569BE
:1091F00076697769786979697A697B6B7C6B7D6B55
:109200007E6B12000301745129E10301270EC56F23
:109210000B0EC66F03011D0EC36F0B0EC46FA0ECC7
:1092200040F000092AE00B01275115E11DCB75F331
:109230001ECB76F31FCB77F320CB78F321CB79F3DA
:1092400022CB7AF323CB7BF324CB7CF325CB7DF3AA
:1092500026CB7EF3010C0301010E746F0301C96B71
:1092600003011D0EC76F0B0EC86F13EC41F0000910
:1092700003E00301746B010C000C010C7FC3E9FFD8
:1092800080C3EAFFEECF23FBEECF24FBEECF25FB1E
:10929000EFCF26FB0301010EC96F03011D0EC76F3F
:1092A0000B0EC86F13EF41F081C3E9FF82C3EAFFE1
:1092B00003017B51EE1808E17C51EE1805E17D5168
:1092C000EE1802E17E51EE1814E00001DF510301B7
:1092D0007B5D20E10001E05103017C5D1BE10001A9
:1092E000E15103017D5D16E10001E25103017E5D64
:1092F00011E183C3E9FF84C3EAFF75C3EEFF76C3C0
:10930000EEFF77C3EEFF78C3EEFF79C3EEFF7AC3BB
:06931000EEFF010C000C51
:0A9316005458540048544D00434CD5
:109320004100435353004A53000047494600434716
:1093300049004A5047004A4152005741560054588C
:1093400054005A5458005A4854005A434C005A4347
:1093500053005A4A5300485454502F312E30203273
:109360003030204F4B00436F6E74656E742D7479EE
:1093700070653A2000436F6E74656E742D456E63A0
:109380006F64696E673A20677A69700D0A004578E4
:1093900070697265733A20300D0A00436163686535
:1093A0002D436F6E74726F6C3A206D61782D61671A
:1093B000653D3330302C206D7573742D7265766188
:1093C0006C69646174650D0A0047455400494E4458
:1093D00045582E48544D004C4F47494E2E4347495F
:0193E000008C
:0E93E2002A0EF66E080EF76E000EF86E0301EE
:1093F0000900F550B46F0900F550B56F03E1B4678B
:1094000001D03DD00900F550AF6F0900F550B06FA5
:109410000900F550B16F09000900F550E96E090027
:10942000F550EA6E090009000900F550B26F090015
:10943000F550B36F09000900F6CFB6F3F7CFB7F3D5
:10944000F8CFB8F3AFC3F6FFB0C3F7FFB1C3F8FF6F
:109450000301B25302E1B35307E00900F550EE6E89
:10946000B207F8E2B307F9D7B6C3F6FFB7C3F7FF01
:10947000B8C3F8FF0301B407000EB55BBFD71200F5
:109480004142434445464748494A4B4C4D4E4F5054
:109490005152535455565758595A61626364656620
:1094A0006768696A6B6C6D6E6F70717273747576D4
:1094B0007778797A303132333435363738392B2F63
:0194C00000AB
:0E94C2003F0EC716C66AC56A0301D351C61213
:1094D000D451C71294869488C68AD5C3C8FF120097
:1094E000C586C7A0FED7C9501200D6C3C9FFC6BEE5
:0894F000FF0CC7B0FED7000C11
:0894F8000301DB51DB07000951
:1095000007E00B010D0E586F5851F6E05807FCD7D5
:1095100012000301DC51DC07000907E0080EE66ECB
:0C952000D6EC4AF0E5520400F4D712002B
:04952C004E6F7420EA
:10953000496D706C656D656E746564006368656324
:109540006B65640064697361626C6564003C212D25
:0D9550002D002D2D3E006F6E006F66660031
:02955E00036A9E
:10956000026A100EE76ED8900636073602360336CA
:109570000B50025C0C50035805E30B50025E0C507C
:0A958000035A062AE72EF0D7120066
:06958A000301CC6BCD6B68
:10959000CE6BCF6BD06BD16B580ED66E9E0ED76E46
:0C95A000010ED56ED58EF284F28A120006
:0495AC00FF0EE3507B
:1095B000246E480E01D04C0EE76EE72EFED7E76A08
:0C95C000E72EFED7242EF7D70000120083
:0495CC0056332E30B4
:1095D0003600415554484F52495A4154494F4E3A2A
:0895E0002042415349432000E1
:0895E800036A080EE76ED8903B
:1095F000073603360C50035C02E3036E072AE72E9E
:04960000F7D7120086
:0C9604001EEE00F02EEE00F0F86A0F9C45
:0C961000F1EC49F007EC3EF0FDD7120031
:04961C0056322E3460
:02962000370011
:049622001200120020
:0296260000043E
:08962800087AF179D579BD79CA
:089630009D797C793D792079D8
:039638000000002F
:02963B0000002D
:03963D000B7901A5
:1096400079ED78E478D478CA780179BF78A67899EA
:10965000780B790B790179ED78E478D47872784BCE
:0396600078EA772E
:0D9663007C2424247D7273747576777879E9
:109670007A7B242424242424243E3F404142434432
:1096800045464748494A4B4C4D4E4F505152535412
:1096900055565724242424242458595A5B5C5D5E73
:1096A0005F606162636465666768696A6B6C6D6E52
:0496B0006F70710066
:0C96B400267B217B1C7B177B127B0D7B2F
:1096C000087BFC7AE47AD47ACA7AC37AAD7A987A3B
:0A96D0007D7A727A5A7A237A1A7AA8
:0496DA0000FF00008D
:0296DE00FFFF8C
:0A96E000BE0FBB0FB80F740F710F1F
:020000040030CA
:0100010046B8
:010002000EEF
:010003000EEE
:010005008377
:010006008178
:01000800FFF8
:010009008076
:01000A00FFF6
:01000B008074
:01000C00FFF4
:01000D0000F2
:0200000400F00A
:100000000A0100010004A3000000FF0000000A0133
:10001000000104012803010A0100010A010001078F
:10002000000700FFFFFFFFFFFFFF000000000000D0
:1000300000032E000061646D696E0000000070779F
:10004000000000000000004D58424F415244202063
:10005000202020202020000A0100016BD36CD30057
:10006000000001000201000000000000000000008C
:1000700000003500500000000000000000000000FB
:100080000000000000000000000000000000000070
:100090000000000000000000000000000000000060
:1000A0000000000000000000000000000000000050
:1000B0000000000000000000000000000000000040
:1000C0000000000000000000000000000000000030
:1000D0000000000000000000000000000000000020
:1000E0000000000000000000000000000000000010
:1000F0000000000000000000000000000000000000
:06010000112233996CD3BB
:00000001FF
